:020000040800F2
:1000000000180020836B0008316B0008F96B0008B2
:10001000356B0008376B0008396B000800000000E2
:100020000000000000000000000000003B6B000822
:100030003D6B0008000000003F6B0008DD0D00086C
:10004000436B0008456B0008476B0008496B0008CC
:100050004B6B00084D6B00084F6B0008516B00089C
:10006000536B0008556B0008576B0008596B00086C
:100070005B6B00085D6B00085F6B0008616B00083C
:10008000636B0008656B0008676B0008696B00080C
:100090006B6B00086D6B00086F6B0008716B0008DC
:1000A000736B0008756B0008776B0008610E000821
:1000B0007B6B00087D6B00087F6B000841620008C5
:1000C0009023DB05802252049A61024B04221A60BD
:0800D0007047C0462015002016
:1000D80033230349034A0A60013B002BFBD17047D5
:0800E80000300040AAAA00004C
:1000F0002E4A91698023DB010B4393619023DB053A
:100100001A682B490A401A601968802292030A4330
:100110001A60284A1168284801401160106880213F
:10012000890101431160596A244801405962586AA3
:100130008021490001435962136A21490B4013622F
:10014000204B214A1360214A1360214B1B68392B35
:1001500027D01CD8132B26D0263B5A1E93415B4236
:100160001C4A13401C4A944663441C4A93818023D2
:100170009B025360002393602C33136013680121AA
:100180000B431360164B802212051A607047603BC8
:100190005A1E93415B42134A1340134A94466344E8
:1001A000E3E7124BE1E7124BDFE7C04600100240E5
:1001B000FFFFEFFF00040048FFEFFFFFFFF0FFFF2E
:1001C000FFFFFFF004110020081500200415002097
:1001D00028150020BFFCFFFFE204000000380140AA
:1001E00000E100E019EEFFFF88130000410300006A
:0401F000C40900003E
:1001F40004498022CB691A42FCD080B2014B188595
:080204007047C04600380140BC
:10020C0010B50400074B1B68002B04D0064B1B6871
:10021C00002B03D110BDFFF7E7FFF7E7200006F036
:0C022C005DF8F7E7101500202C140020EE
:1002380010B50400454B1868C343454A1168CA43C2
:100248000140013100D170E0424901200860190CD9
:10025800414801601B041B0C40480360002902D17F
:100268003D493F480860002B02D13C4B3D4919608D
:10027800D107C91706230B400A333B490B603B499A
:100288000B6013065B0E3A490B60002C4CD05305EB
:100298009B0F38490B601304DB0E043336490B609F
:1002A800120C364B1A60364B1A68D24313041B0CD7
:1002B80034490B60120C344B1A60344B1B68DB4317
:1002C8001B041B0C802109018B4201D930490B43C7
:1002D80030490B60002A2DD12F4B304C304819196A
:1002E80004CBD2430A608342F9D12E4C2E48191907
:1002F80004CBD2430A608342F9D103F031FF214B8A
:100308001B68002B07D09023DB051B8A5B0502D4F2
:100318001C4B00221A600D20FFF774FF04F0E2FA6C
:10032800184B1B68002B0AD110BD04F0F5F8002CFF
:10033800E3D1F9E702F0EEFA02F04CFBCCE7013B1F
:100348001A4A136003F01AFCEEE7C046007400086E
:100358000474000818150020C41400201C1500207F
:10036800830400004057000084140020501400202B
:100378002815002060140020681400206414002050
:1003880008740008C01400209C1400200C74000895
:100398000000FFFF80140020107400080094FF176D
:1003A800007A00081088FF17008000087C140020DD
:1003B800F0B5C64600B586B001A9294B0A0013CB93
:1003C80013C203CB03C2274B01221A60264B00221B
:1003D8001A6005F073F9254A254B1A60254B984693
:1003E800254F234E254D06E02B68002B13D1204BBB
:1003F8001B68002B0FD043461F6034689442F3D02B
:10040800A3059B0D1E4922008B42EDD12E20FFF73C
:10041800F9FE2200E8E701A806F00FFC174B1B685D
:10042800002B0CD06F20FFF7EDFE6B20FFF7EAFEE4
:10043800C82000F089F806B080BCB846F0BD652039
:10044800FFF7E0FE7220FFF7DDFE7220FFF7DAFE0D
:100458006F20FFF7D7FE7220FFF7D4FEE8E7C0460B
:1004680070630008C814002028140020B80B00008E
:100478000C15002000300040AAAA00002C1400200F
:04048800FF0300006E
:10048C0010B5254B1B68002B22D1234B32221A604E
:10049C00224B234A1A60234B1B68002B19D0013BBB
:1004AC00204A1360002B14D09023DB051B8A9B057C
:1004BC000ED51D4B1B68002B0AD01C4B1B68002B48
:1004CC0006D01B4B1B685A1C132B08D0184B1A60F8
:1004DC0010BD9023DB05802252009A61E4E7144B97
:1004EC0000221A60134B1B68002BF1D1124B1A60BF
:1004FC00124B1B681F2B09D0114B1B68002BE7D12B
:10050C00FFF754FF0D20FFF77BFEE1E70B4B0B329F
:10051C001A60FFF7E7FDEFE71415002000300040EC
:10052C00AAAA000020150020C41400201C150020CD
:10053C00101400202C140020101500202815002069
:04054C00C8140020AF
:1005500010B5054B1860002805D01C00FFF796FF6A
:0C0560002368002BFAD110BD24150020E8
:10056C00F8B5D0490122CB681A42FCD1CD4B1B699E
:10057C001B0604D5CB4BCC4A5A60CC4A5A60C94BAB
:10058C001A6902210A431A61C94A5A611A693E3131
:10059C000A431A6119000122CB681A42FCD1C14BE3
:1005AC00DB689B0604D5BF4AD36820210B43D3607C
:1005BC00BC4B1A6902218A431A611A6901390A4330
:1005CC001A61BC4B1B68DB43B94A1380B549012245
:1005DC00CB681A42FCD1B34BDB689B0604D5B14AFD
:1005EC00D36820210B43D360B34B1B68DB43B34A66
:1005FC001380AC490122CB681A42FCD1A94BDB68B1
:10060C009B0604D5A74AD36820210B43D360AC4B7F
:10061C001B685B00FF221A40AA4B1B680A3B591E41
:10062C008B411A43A84B1B685B02C021C9000B40CD
:10063C001A43A64B1B68043BDB061B0C1343DB4322
:10064C00A34A138097490122CB681A42FCD1954BDF
:10065C00DB689B0604D5934AD36820210B43D360F7
:10066C009C4B1B68DB439C4A13808E490122CB6850
:10067C001A42FCD18B4BDB689B0604D5894AD368A4
:10068C0020210B43D360954B1B68DB43944A1380AA
:10069C0084490122CB681A42FCD1824BDB689B0651
:1006AC0004D5804AD36820210B43D3608D4B1B6843
:1006BC00DB438D4A13807B490122CB681A42FCD163
:1006CC00784BDB689B0604D5764AD36820210B4314
:1006DC00D360864B1B68DB43854A1380714901222A
:1006EC00CB681A42FCD16F4BDB689B0604D56D4A74
:1006FC00D36820210B43D3607E4B012252421A80D7
:10070C0068490232CB681A42FCD1664BDB689B0607
:10071C0004D5644AD36820210B43D3607648774CC8
:10072C00241A604B01222025754F02E00430B84298
:10073C001AD006190168C9433180D9680A42FCD124
:10074C00D9680D4202D0D9682943D9600168C943E0
:10075C00090C7180D9680A42FCD1D9680D42E5D0E8
:10076C00D9682943D960E1E74E4B1A6901218A43C4
:10077C001A61644A644911601A6902210A431A61B8
:10078C00624A5A611A693E310A431A611900012200
:10079C00CB681A42FCD1434BDB689B0604D5414A1B
:1007AC00D36820210B43D3603E4B1A6902218A4344
:1007BC001A611A6901390A431A615148012220252C
:1007CC00534F02E00430B8421AD006190168C943ED
:1007DC003180D9680A42FCD1D9680D4202D0D9685F
:1007EC002943D9600168C943090C7180D9680A4250
:1007FC00FCD1D9680D42E5D0D9682943D960E1E72D
:10080C004448454C241A274B01222025434F02E033
:10081C000430B84219D006190168C9433180D9682F
:10082C000A42FCD1D9680D4202D0D9682943D9605B
:10083C004188C9437180D9680A42FCD1D9680D42FC
:10084C00E6D0D9682943D960E2E7164B1A69012131
:10085C008A431A612B4A2C4911601A6902210A43F6
:10086C001A612F4A5A611A693E310A431A611900FA
:10087C000122CB681A42FCD10A4BDB689B0604D5DB
:10088C00084AD36820210B43D360064B1A69022116
:10089C008A431A611A6901390A431A610122202517
:1008AC00204F44E00020024023016745AB89EFCD87
:1008BC00007400081C150020C414002002740008E9
:1008CC0028150020841400206014002068140020D7
:1008DC00047400086414002006740008C01400207E
:1008EC00087400089C1400200A740008801400206E
:1008FC000C7400080E740008100800201074000816
:10090C00000C002000300040AAAA0000007800086B
:10091C00000E002010020020007A000810040020B5
:10092C00007C0008100800200430B84219D00619C9
:10093C000168C9433180D9680A42FCD1D9680D429B
:10094C0002D0D9682943D9604188C9437180D968DC
:10095C000A42FCD1D9680D42E6D0D9682943D96046
:10096C00E2E7064B1A6901218A431A611A697F3141
:10097C000A431A610A20FFF7E5FDF8BD002002408A
:10098C0070B5041E00DA9CE0092C00D893E0632CAF
:10099C0000D881E0FA239B009C426ED3534B9C42BF
:1009AC005AD9534B9C4248D9524B9C4236D9524B44
:1009BC009C4224D9514B9C4212D9514B9C4200D998
:1009CC0084E05049200006F0ACFB05004D492000A6
:1009DC0006F032FB0C0028003030C0B2FFF710FCE0
:1009EC004949200006F09DFB05004749200006F010
:1009FC0023FB0C0028003030C0B2FFF701FC434948
:100A0C00200006F08EFB05004049200006F014FB88
:100A1C000C0028003030C0B2FFF7F2FB3C4920003C
:100A2C0006F07FFB05003A49200006F005FB0C00A0
:100A3C0028003030C0B2FFF7E3FB3649200006F047
:100A4C0070FB05003349200006F0F6FA0C00280074
:100A5C003030C0B2FFF7D4FBFA218900200006F039
:100A6C0060FB0500FA218900200006F0E5FA0C0075
:100A7C0028003030C0B2FFF7C3FB6421200006F021
:100A8C0050FB05006421200006F0D6FA0C0028006B
:100A9C003030C0B2FFF7B4FB0A21200006F041FB56
:100AAC0005000A21200006F0C7FA0C00280030309F
:100ABC00C0B2FFF7A5FB20003030C0B2FFF7A0FB9F
:100ACC0070BD2D20FFF79CFB64425DE712492000AE
:100ADC0006F027FB05001049200006F0ADFA0C00CB
:100AEC0028003030C0B2FFF78BFB6AE70F270000FD
:100AFC009F8601003F420F007F969800FFE0F505AE
:100B0C00FFC99A3B00E1F5058096980040420F0022
:0C0B1C00A08601001027000000CA9A3BD0
:100B280070B58CB006AD124B2A0013CB13C213CB91
:100B380013C26C460F4B220043CB43C243CB43C284
:100B48000D20FFF75FFB280006F077F83520FFF748
:100B580059FB2E20FFF756FB2420FFF713FF200038
:100B680006F06BF80D20FFF74DFB0CB070BDC046CA
:080B7800846300089C6300087F
:100B800010B5544B5969802292020A435A6159693F
:100B90008022D2020A435A619022D20500231360B8
:100BA0004D490B604D48D0604D48C860D0684D4CF1
:100BB0002040D060116821401160106880214902F6
:100BC00001431160802149009161474ACE3911608B
:100BD000464A1360464A1360464A1360464A4749EC
:100BE0001160474A47491160474A1360474A1360FA
:100BF000474A13600A2247490A6047490A60474A40
:100C00001360474B0B221A60464B474A1A60474B0A
:100C10001868FA21890006F08AFA013880235B04FB
:100C200098420DD2424A50604248036A1B021B0A96
:100C3000C02109060B43036200239360073313604E
:100C40000A20FFF785FC3C4C3C4B23603C4BA360E7
:100C50000220FFF77DFC022363600220FFF778FC8F
:100C6000384B23600020FFF7E7FA0220FFF770FC03
:100C7000FFF73EFA0220FFF76BFCFFF755FF02205B
:100C8000FFF766FC304B00221A609023DB051B8ABD
:100C90009B0507D5184B1B68002B03D0184B1B680E
:100CA000934213D1294805F0CCFF0D20FFF7A2FA9B
:100CB0000120FFF7C1FA264C03F0BEFA01F06EFFE7
:100CC0002368002BF8D002F0C1FFF5E7FFF774FBB3
:100CD000EEE7C0460010024000040048AAAA0AA499
:100CE000AAAAAAAAFFFFFCFF1415002020150020C5
:100CF000241500200C150020C414002083040000DB
:100D00001C1500204057000028140020C8140020A3
:100D10001815002084140020501400201015002005
:100D20002815002074140020A1B0B9120C02002074
:100D300010E000E000ED00E00030004055550000FC
:100D4000FFFF0000CCCC00002C140020E06F000856
:040D50004414002027
:100D540010B5FFF799FB0F4B1B680F4A12689342BB
:100D640016D05A1C0B490A601B78802000021843D5
:100D74000A4B1B689A4208D09023DB058022520458
:100D84009A61074B04221A6010BD064A0A60F3E711
:100D94000020F9E7041500200815002008020020AF
:080DA4002015002004110020BD
:100DAC0010B5094B1B68002B05D1084B1B680020A4
:100DBC00002B05D010BD05F073F80028F5D0F9E72D
:100DCC00FFF7C2FFF6E7C0462C14002010150020D8
:100DDC00194B1B68002B02D0013B174A1360174BB1
:100DEC001B68002B02D0013B144A1360144B1B6888
:100DFC00002B02D0013B124A1360124B1B68002BD4
:100E0C0002D0013B0F4A13600F4B1B68002B02D022
:100E1C00013B0D4A13600D4B1B68002B02D0013BAC
:100E2C000A4A13600A490A6853035A40530C534048
:100E3C005A0153400B6070471415002024150020F4
:100E4C000C15002090140020541400206C14002069
:040E5C0074140020EA
:100E600010B51A4BDB699B062BD5184B9B8C9BB29C
:100E7000174A1268002A1AD1FF321A40022A0FD0EC
:100E8000042A11D0134A11680B70136801331360E0
:100E9000114A1268934214D10E4B104A1A6010E0A6
:100EA0000F4A02211160EDE700F052FD09E0094A06
:100EB00011680B70136801331360074A126893427C
:100EC00000D010BD034B054A1A60FAE70038014014
:100ED0001015002008150020080200200411002031
:040EE0004814002092
:100EE400024A202311680B4313607047A0140020AA
:100EF400064A1368043B1360054A0C32934204D239
:100F0400044A042311680B431360704770140020D3
:080F14005C130020A014002072
:100F1C00084B1A68111D1960074B5433994202D2C1
:100F2C00136853607047054A042311680B43136020
:100F3C00F8E7C046701400205C130020A0140020B9
:100F4C00044B19680A1F1068096811601B68186047
:080F5C007047C046701400202C
:100F6400034A1368191D11601A1F12685A607047EA
:040F740070140020D5
:100F7800074A1368190008390868043B1B680B60A6
:100F88001368191F1B680B60136818607047C04608
:040F980070140020B1
:100F9C00074A13681968181F006818601368181F2F
:100FAC00083B1B6803601368083B19607047C04618
:040FBC00701400208D
:100FC0000C4B19680A680C4BCB1A9B109B1A042B0C
:100FD00006D4002A0AD092008A1A13680B60704760
:100FE000064A042311680B431360F8E70439014BE8
:100FF0001960F4E7701400205C130020A014002096
:1010000030B5144B1A681168134BD31A9B105B1A36
:10101000042B19D4043A0F4B1A60012913D9012368
:101020005B1A9B009D580222521A9200094C2368B9
:1010300098589B18043B1860013904320029F6D1F6
:10104000044B1B681D6030BD044A042311680B4328
:101050001360F8E7701400205C130020A014002037
:10106000F0B5144B1A681568134BD31A9B105B1B11
:10107000042B19D4043A17680E4B1A60012D12D9AB
:101080006E1E0422524200211C00236898589B18AF
:1010900058600131043AB142F7D101235D1B054B81
:1010A0001B68AD00EF50F0BD044A042311680B43E8
:1010B0001360F8E7701400205C130020A0140020D7
:1010C000054B1A68111F12680868844662440A605A
:0C10D0001A68043A1A607047701400207F
:1010DC00024B1A68136801331360704770140020B8
:1010EC00054B1A68111F12680868821A0A601A6880
:0C10FC00043A1A607047C04670140020CF
:10110800024B1A681368013B136070477014002083
:10111800044B1A681368002B00DB70475B421360AE
:08112800FBE7C0467014002033
:1011300010B50F4B1B681A68D117501848401F286C
:1011400009DC191F0A4C2160002A0BDB0B0009681F
:101150009140196010BD074A8023DB0011680B43E2
:101160001360F7E7043B1A68C2401A60F2E7C04612
:0811700070140020A0140020FF
:10117800054B1A68111F1268086802400A601A684D
:0C118800043A1A607047C0467014002042
:10119400054B1A68111F1268086802430A601A682E
:0C11A400043A1A607047C0467014002026
:1011B000054B1A68111F1268086842400A601A68D5
:0C11C000043A1A607047C046701400200A
:1011CC00024B1A681368DB431360704770140020DD
:1011DC00024B1A6813685B4213607047701400204E
:1011EC00054B1A68111F1268086842430A601A6896
:0C11FC00043A1A607047C04670140020CE
:1012080010B50B4B1C682168002909D0043C2068E4
:1012180005F06BFF2060064A1368043B136010BD9D
:10122800044A80231B0111680B431360F7E7C0468B
:0812380070140020A014002036
:1012400010B50B4B1C68216800290AD0221F1068BA
:10125000083C23685843064B1C6005F04AFF206099
:1012600010BD044A80231B0111680B431360F7E78C
:0812700070140020A0140020FE
:1012780010B50B4B1C682168002909D0043C206874
:1012880005F065FF2160064A1368043B136010BD32
:10129800044A80231B0111680B431360F7E7C0461B
:0812A80070140020A0140020C6
:1012B00070B50D4B1C682568002D0ED0043C2668C7
:1012C0002900300005F047FF2160074B1C6829000A
:1012D000300005F00EFF206070BD044A80231B0122
:1012E00011680B431360F7E770140020A01400206E
:1012F000034A1368191D1160024A12685A60704748
:08130000701400207414002099
:10130800064A1368191F1B6808681B1A584243418C
:101318000B601368043B13607047C04670140020CC
:10132800064A1368191F1B6808681B1A581E834150
:101338000B601368043B13607047C04670140020AC
:10134800034B1A6811684B424B4113607047C04603
:0413580070140020ED
:10135C00074B1A68131F012112681868904200DCB1
:10136C0000211960024A1368043B13607047C046A1
:04137C0070140020C9
:1013800030B5074B1A68111F10680A68D217C40FCE
:101390000D68854262410A601A68043A1A6030BDDD
:0413A00070140020A5
:1013A400074B1A68131F012112681868904200DB6A
:1013B40000211960024A1368043B13607047C04659
:0413C4007014002081
:1013C800064A1368191F1B68086884469C459B4198
:1013D8005B420B601368043B136070477014002075
:1013E80030B5074B1A68111F08681468C20FE51753
:1013F80084426A410A601A68043A1A6030BDC046DD
:04140800701400203C
:10140C00044B0A221A60044B1B68002B01D1034BBE
:10141C001A60704750140020A4140020841400207B
:10142C00044B10221A60044B1B68002B01D1034B98
:10143C001A60704750140020A4140020841400205B
:10144C000F4B1B68012B05D00E4A402311680B4330
:10145C00136070470C4B19680A1D1A600B4B1B6804
:10146C000B4A1268934203D005D2D31A4B60F0E7B3
:10147C0000234B60EDE79B1AC4334B60E9E7C04691
:10148C0010150020A014002070140020041500205A
:04149C00081500200F
:1014A00006490A681368043A0A60002B05D004490B
:1014B000044A0A60013B002BFBD1704770140020E6
:0814C00000300040AAAA000060
:1014C80004490B6864221868424303480260043BDD
:0C14D8000B6070477014002054140020BA
:1014E40010B5054B1C68221D1A60044B1868642152
:1014F40005F01BFE606010BD701400205414002021
:1015040030B5094B1B68013B08495B181B041C0CD4
:10151400074802681B0E15684B5513689C466144C6
:101524004C70043A026030BDB01400201002002058
:04153400701400200F
:10153800044B1A68111D1960034B1B68043B1B6898
:0C154800536070477014002078140020DD
:10155400024B1B681A68024B1A607047781400200B
:0415640098140020B7
:10156800064B1B681A68002A04D1054A12681168DC
:10157800044A1160043B014A13607047701400204C
:081588007814002098140020E3
:10159000154B1B68154A19681160154A934218D9F2
:1015A000144A1268022A07D0043B0F4A1360124AF9
:1015B0001368013B136070470F4A11680F4A1268A5
:1015C0009142F1D10D4A002111600A4A03311160A4
:1015D000EAE7064B00221A60064B1B68022BEAD191
:1015E000044B03321A60E6E77814002098140020B8
:1015F000F8120020FC0100208C140020BC140020F4
:10160000054B00221A605A609A6018000C3003499A
:101610000860DA607047C0465C1300207014002038
:0C162000014B03221A607047FC010020FF
:0C162C00014B01221A607047FC010020F5
:0C163800014B00221A607047FC010020EA
:1016440030B50D4B1C68221D1A600C490B685A1CDE
:101654000A60587800069A1C0A609A7812040243B9
:10166400D81C0860D87800021D1D0D601B79134337
:101674000343636030BDC0467014002098140020FA
:10168400054A1368191D116004490A68501C086052
:1016940052785A607047C046701400209814002095
:1016A400074B19680A1D1A60064A1368581C106013
:1016B4005A781201044B9B189B684B607047C046D4
:0C16C40070140020981400201008002072
:1016D000074B1A68511C19600648036851780901C4
:1016E000054A521819689160043B03607047C04670
:0C16F00098140020701400201008002046
:1016FC00074B1A68511C196051780902901C18602C
:10170C0092781143802292050A431A607047C046B2
:04171C0098140020FD
:1017200010B5094B1868021D1A6008490B685A1C4D
:101730000A605A7812029C1C0C609B781A43802322
:101740009B051343436010BD7814002098140020BB
:10175000084B094A1A60094B1A68511C19605178E4
:101760000902901C186092781143802292050A4366
:101770001A60704700300040AAAA000098140020A8
:1017800010B5094B1B681A68023A80239B05134366
:101790001A78752A03D1013B044A136010BD034A2D
:1017A0001360FFF7D5FFF9E77814002098140020A4
:1017B00010B50A4B1B681B68002B0CD0084A136835
:1017C000043B1360074A136803331360034A13682A
:1017D000043B136010BDFFF7BBFFF7E77014002058
:0817E000781400209814002089
:1017E80010B50A4B1B681B68002B0CD1084A1368FC
:1017F800043B1360074A136803331360034A1368F2
:10180800043B136010BDFFF79FFFF7E7701400203B
:08181800781400209814002050
:1018200010B5104B1A681100103119600E490B6881
:10183000180008380068D060181F006890601868A9
:1018400050600C3B0B6009480368591C01605978D3
:1018500009029C1C04609B78194380239B050B4361
:10186000136110BD7814002070140020981400201B
:1018700010B5254B1B681A1F126819000839086833
:101880000C3B19685318214A214C146000291DDBB8
:10189000984212DD1C4A1268043A13601D4B1A6804
:1018A000511C196051780902901C186092781143FC
:1018B000802292050A431A6010BD134A1368103B38
:1018C0001360144A136803331360F5E7984212DA81
:1018D0000D4A1268043A13600E4B1A68511C1960C5
:1018E00051780902901C1860927811438022920569
:1018F0000A431A60E0E7044A1368103B1360054A84
:10190000136803331360D7E77814002000300040D9
:08191000AAAA000098140020AF
:10191800024A1368043B13607047C04678140020DD
:10192800024A1368103B13607047C04678140020C1
:1019380010B5044C23681878FEF764FC2368043B50
:08194800236010BD70140020A3
:1019500000B583B06A46094B03CB03C2084B1B6832
:10196000002B01D003B000BD684605F06AF9044BB6
:1019700001221A60034B00221A60F3E7B4630008E7
:08198000FC01002048140020C6
:1019880010B5114B1B68002B12D0104B1B78002B85
:101998000ED00F4B1B68002B15D00E4A1368191D6B
:1019A80011600D4A12785A60094B00221A600AE049
:1019B800FFF7F8F90028FBD0064B1A68111D1960CB
:1019C800FF231840506010BDFC0100203315002093
:0C19D8004C140020701400203215002078
:1019E40010B50E4B1B68102B08D00D4B1B681868E4
:1019F400E0231B06C2180B4B9A420CD8084B1B68F9
:101A0400186805F068FB2020FEF7FEFB044A136803
:101A1400043B136010BDFEF7B7FFF4E75014002039
:081A240070140020FF0B0630D6
:101A2C0010B5064C2368186805F051FB2020FEF712
:101A3C00E7FB2368043B236010BDC04670140020F4
:101A4C00F0B587B003AA2A4B13CB13C2294B1A68E3
:101A5C0001929A8801AB9A805B20FEF7D1FB264B52
:101A6C001B68264A0C3293420DD0244A0C32934206
:101A7C000DD3224A0C32934216D9204C1034042533
:101A8C001E4F160024E001A805F0D5F80CE003A8C1
:101A9C0005F0D1F8194B00221A605A609A601800B0
:101AAC000C3015490860DA605D20FEF7A9FB202098
:101ABC00FEF7A6FB07B0F0BD206805F008FB202060
:101ACC00FEF79EFB01350C4B1B680434B342EBD97B
:101ADC00DB1B9B10AB42E7D32020FEF791FB084B9E
:101AEC001B68102BE8D02068FEF74AFFE7E7C046DA
:101AFC00146C0008206C0008701400205C1300208B
:041B0C005014002051
:101B1000F0B5D6464F464646C0B584B001AA394B0B
:101B200003CB03C21B7813702020FEF76FFB364BEC
:101B30001B68002B5BD0354D00270026C0231B05FA
:101B40009946334B9A46304B984616E02020FEF7D4
:101B50005DFB14E06B684A46134221D12020FEF75A
:101B600055FB2020FEF752FB01360137052F34D8F4
:101B7000103543461B68B34237D9092EE6D93000E9
:101B8000FEF704FF3A20FEF741FB2C00083C2078CA
:101B90000028DFD0FEF73AFB0134AC42F7D1D9E799
:101BA00001A805F04EF853461B68102B11D0286889
:101BB000FEF7ECFE2020FEF729FB4020FEF726FB77
:101BC0002804000C05F089FA2920FEF71FFB0237D4
:101BD000C4E7286805F081FAECE70D20FEF716FB54
:101BE0002020FEF713FB0027C2E7002F05D104B029
:101BF000E0BCBA46B146A846F0BD0D20FEF706FB94
:101C0000F5E7C046786E0008881400201808002008
:041C1000501400204C
:101C140010B5044C2368186805F0BFF82368043B2A
:081C2400236010BD70140020C4
:101C2C0010B5074B1B68002B04D1064A1368043B04
:101C3C00136010BD034B1B681878FEF7D5FAF4E758
:081C4C001015002070140020A7
:101C5400F0B5C64600B5114A13681F68043B13600B
:101C6400002F13D00125ED1BAD003C000C4E904617
:101C740003E0013C0435002C08D03368002BF8D075
:101C840043461B68585DFEF7B3FAF2E7034BBF0007
:101C94001A68D71B1F6080BCB846F0BD70140020C2
:041CA40010150020F7
:101CA800F0B5C64600B582B06846214B020012CB9B
:101CB80012C204F0C2FF0D20FEF7A4FA1D4DFC234A
:101CC8009B009846A8440026012723E0FEF79AFACD
:101CD8000134285D0028F9D1062C05D82020FEF70C
:101CE80091FA0134072CF9D12320FEF78BFA38003A
:101CF80004F0CBFF2020FEF785FA2020FEF782FAB9
:101D08002020FEF77FFA01370136052E07D0083567
:101D1800A84509D02020FEF775FA0024D9E70D2040
:101D2800FEF770FA0026F2E702B080BCB846F0BDB4
:081D3800BC63000828670008E5
:101D400070B5FFF733F8041E00D1D8E0C0B2704B75
:101D50001B68002B08D06F4B1B78002B04D06E4BF8
:101D600018706E4B01221A600A2800D1C4E00228C4
:101D700000D8C3E0674B1B78002B08D109281FD07F
:101D8000674A12683F2A02D9202800D19EE02828FD
:101D900018D02F2840D01B2868D10024002B00D158
:101DA000ADE00E38FEF732FA5D4B1A685D4B20212C
:101DB00099549B18002159705B4B1A6002349EE0C5
:101DC0001730DDE7594B1C68002C01D0002496E049
:101DD000FEF71CFAFEF7EAFF0028FBD0C0B220286D
:101DE0000BD04F490B684F4A2825D554D218507054
:101DF00002330B60FEF70AFA81E0494B1B6801339E
:101E00004A4A13601838FEF701FA2020FEF7FEF95F
:101E10000820FEF7FBF972E0444B1C68002C01D04F
:101E200000246CE0FEF7F2F9FEF7C0FF0028FBD0BB
:101E3000C0B22F280BD03A490B683A4A2F25D55407
:101E4000D218507002330B60FEF7E0F957E0344BC4
:101E50001B680133354A13602738FEF7D7F9202075
:101E6000FEF7D4F90820FEF7D1F948E0092848D058
:101E7000122848D0082817D12C4B1D680024002DAB
:101E80003DD1274B1C68002C39D0013C1C60254BF0
:101E900020221A55FEF7BAF92020FEF7B7F90820DC
:101EA000FEF7B4F92C002AE00D2817D11C4B1B6853
:101EB000002B0BD11A4B1A681A4B202199549B18EE
:101EC00000215970184B1A60012418E0174B1B6849
:101ED000012BEFD00D20FEF799F9EBE7134B1C68AF
:101EE000002C12D10E4D0F4B2A689854FEF78EF934
:101EF0002B6801332B6002E0002400E00024200066
:101F000070BD0324FBE70424F9E70024F7E7C0468B
:101F1000FC01002033150020321500204C14002055
:101F2000401400209412002044140020A814002023
:101F300010B5154B1968154B5A5C202A09D14B1C5A
:101F40001248013819000133C25C202AFAD00E4B26
:101F500019600023002A10D00C4840180C4CC25CB9
:101F6000202A03D01A5501330F2BF8D1084A00203C
:101F7000D0545B18074A136010BD054B00221A703D
:101F8000044B1960F8E7C046381400209412002072
:081F9000C013002040140020E2
:101F9800F0B5DE46474680B587B00E0002AA002499
:101FA80005E0002B1BD001340132102C08D0035D52
:101FB8001370190061391929F3D8203B1370F2E71F
:101FC800002302AAD37313782D2B0ED1254B0022A0
:101FD8001A6001239B460127012C0FD82CE000230F
:101FE80002AAD37313782D2B2CD01E4B00221A6013
:101FF80000239B4600270120002C2DD0194B1D687B
:10200800B84602AB9C46E044002301934346187847
:10201800310004F0CCFE431C18D075432D1801374D
:1020280001239C46E0440193A742EFD30D4B1D606A
:1020380001205B46002B0FD00A4A13685B421360ED
:10204800012009E00020012CC0D105E0019B002BF4
:1020580001D0044B1D60002007B0C0BCBB46B04691
:08206800F0BDC0463C1400204D
:1020700010B5344B187800285AD000233149013369
:102080005A5C002AFBD12D280FD0302829D12D4AA7
:10209000527820218A43582A11D02B4A11681029DE
:1020A0003AD1082B48D900204BE0012B3AD0264AE0
:1020B000116810292AD00B2B3ED9002041E0214A7B
:1020C00092782D2A09D00A2B2ED81E4810210230D2
:1020D000FFF762FF431E984133E00B2BF5D9002038
:1020E0002FE02528D9D1174A52782D2A09D00B2B59
:1020F0001CD814480A210130FFF74EFF431E9841B7
:102100001FE00C2BF5D900201BE000232D28C8D19F
:10211000092B11D9002014E02D28CCD000200A2B47
:102120000FD809E000200CE000200AE0002008E0C1
:10213000054B19681029E8D00248FFF72DFF431E10
:0C214000984110BDC01300205014002076
:10214C00F0B51A4C00251A4E0021635C8A5D18000C
:10215C00613819280DD8203BDBB2100061381928E2
:10216C0011D8203AD2B2934219D101310829ECD1BD
:10217C0015E01000613819280DD918002038471EB9
:10218C00B84140420340934209D1002AEDD1094B9A
:10219C001D600120F0BD203AD2B2202BE3D10135D5
:1021AC0008347F2DD0D10020F4E7C046206700080A
:0821BC00C01300207C14002078
:1021C40070B51A4B1B78002B29D0194A00231E0026
:1021D400013310321100103909780029F7D1731C2A
:1021E4001FD03301114C1C19124D16E08B4211D132
:1021F40000290BD00132082A0CD0A15C535D1800D1
:1022040061381928F2D8203BDBB2EFE70A4B1E6095
:10221400012070BD103C013E05D30022EDE70020F3
:10222400F7E70020F5E70020F3E7C0461008002098
:0C22340020080020C01300207C140020B3
:1022400010B50F4B1A680F4B1A60FFF771FEFFF7BE
:10225000B9FF002805D00C4B1B6801330B4A1360F3
:1022600010BD0B4B1B78302B05D00A4A2123116877
:102270000B431360F4E7054B00221A60F0E7C046F9
:1022800040140020381400207C140020C0140020CA
:08229000C0130020A01400207F
:10229800074A13680749C85401331360064A934232
:1022A80004D9064A202311680B4313607047C046BF
:1022B800B014002010020020FE050000A014002029
:1022C80010B5144B18688200134BD3581A030AD45C
:1022D800124A1268002A13D19B030BD48000104BBA
:1022E800C358984705E00F4A80239B0011680B43A9
:1022F800136010BD0B4A082311680B431360F8E7FD
:10230800DB0304D58000064BC3589847F1E7FFF775
:10231800BFFFEEE77C14002024650008A414002009
:0823280000000020A0140020B9
:1023300070B594B00CA9414B0A0013CB13C213CB58
:1023400013C203CB03C205A93D4B0A0013CB13C232
:1023500013CB13C21B7813706A463A4B13CB13C2CC
:1023600011001A680A601B790B71374B1B68522BDE
:1023700009D95224354E344DA05DFDF747FF013495
:102380002B68A342F8D85223314A1360314A002106
:102390001160314A13602E4D304E03E02C4B1A6809
:1023A0002D4B1A60284C2B682268934234D2FFF7D9
:1023B000BFFD3378002BF6D0FFF75AFE00280BD074
:1023C000274B1A68274B1A60274B1B78002BE5D048
:1023D000264B01221A60E1E7FFF7B8FE002811D072
:1023E000234B1B689B00234A9B585B0321D5FFF7B7
:1023F0006BFF214B1B68002B08D1154B1A68164B3D
:102400001A60CFE70CA804F01CFC05E01A4B002270
:102410001A60684604F015FC0D20FDF7F7FE522304
:10242000094A13600A4A13600A4B00221A6014B06A
:1024300070BD05A804F005FCEEE7C046906E0008EC
:10244000B06E0008CC6E00084414002094120020E6
:1024500040140020A814002038140020C0130020CD
:102460003C140020B414002033150020B8140020C0
:0C2470007C14002024650008A01400204B
:10247C0070B56F20FFF70AFF0C4D2C68FF20FFF79B
:10248C0005FFFF20FFF702FF2B68013B084A9B1852
:10249C001B04180C074909681B0E0D6853550B6873
:1024AC009C46624450700C6070BDC046B014002055
:0824BC00100200207014002042
:1024C40010B57020FFF7E6FE064A1368191D116067
:1024D400054A12685A60FF20FFF7DCFEFF20FFF771
:0C24E400D9FE10BD70140020B0140020C0
:1024F00010B57420FFF7D0FE064A1368191D11604D
:10250000054A12685A60FF20FFF7C6FEFF20FFF75A
:0C251000C3FE10BD70140020B0140020A9
:10251C00F8B57520FFF7BAFE104E33681D6801350B
:10252C000F4C2D19280AFF273840FFF7AFFE380053
:10253C002840FFF7ABFE0B4B1B68013B1B193268A5
:10254C00190A106821541268A41863707720FFF7D9
:10255C009DFE3368043B3360F8BDC0467014002008
:08256C0010020020B014002051
:1025740010B50E4B1B68002B15D06420FFF78AFEA4
:1025840000220A4B1A600A490B6801330B601B01D5
:1025940008495A54084B1A68084B1A60084B1A68C1
:1025A400084B1A6010BDFEF7F1FFF7E7A4140020F2
:1025B4008814002010080020B0140020AC1400205F
:0825C4008414002050140020D3
:1025CC0070B5324B1B68002B27D1314B1B681C7824
:1025DC0023005F3B022B16D97D20FDF711FE202036
:1025EC00FDF70EFEFFF72CFA2500703D072D15D9CF
:1025FC00743C012C1CD9032D0FD8264B1B68188852
:10260C0004F02FFD09E0244B186801300005000D83
:10261C0004F027FD2920FDF7F3FD70BD2020FDF708
:10262C00EFFD5220FDF7ECFD3A20FDF7E9FDDFE769
:10263C00184B1A68194BD31A082BEED90C3A108880
:10264C0004F00FFD2020FDF7DBFD2020FDF7D8FD69
:10265C00104C2368083B188804F003FD2020FDF77C
:10266C00CFFD6920FDF7CCFD2368043B188804F0EE
:10267C00F8FC2020FDF7C4FD7820FDF7C1FD236890
:10268C001888013004F0EDFCC7E7C046A014002008
:10269C00941400207814002098140020F8120020C4
:1026AC00104B1B68002B0BD00F4B18680F4B1B6883
:1026BC00984205D001D2181A13E0C01AC43010E0A9
:1026CC000B4B186800280BD10A4B1B680A4A12687E
:1026DC00934206D0D01A934203D3981AC43000E028
:1026EC00002070472C140020D4140020D814002093
:0C26FC0010150020041500200815002017
:1027080010B5094B1C68221D1A60084B1B68002B6A
:1027180006D0074B1B78002B02D0064B186801E047
:10272800FFF7C0FF606010BD70140020FC0100209E
:08273800331500204C140020B1
:1027400010B50B4B1C6800230A4909190A48CA5CDA
:10275000222A03D01A5401334E2BF8D1064A2221E3
:10276000D15401330021D154E318044A136010BD41
:102770003814002094120020C013002040140020C0
:102780001A4B1B185A781300613B192B03D8203AB7
:102790001300373B05E02F2A1BD91300303B092BD0
:1027A000F6D80F2B18D8114A101882781100613909
:1027B000192907D8203A373A11000F2912D81801E1
:1027C000401870472F2A0AD9110030390929F4D945
:1027D000F1E701204042F4E701204042F1E7012007
:1027E0004042EEE701204042EBE7C046C013002024
:1027F000F0B5C64600B50700404B1B680133404AA0
:102800001360FFF79DFF002600243E4A03E00136D7
:102810000134502C10D0A35C5C2BF8D0222BF7D1C4
:10282000384B00221A55384B1D68002D0CD1354C01
:10283000364B98461E003BE0354A022311680B4395
:10284000136080BCB846F0BD012F0ED06620FFF7A4
:1028500023FD304A13687600A41B2F49CC54013362
:1028600013600024274D2E0009E06520FFF714FDBA
:10287000EFE7FFF711FD0134335D002BE1D0285D58
:102880005C28F6D12000FFF77BFF431C03D0033404
:10289000FFF702FDF0E71E4A022311680B431360A5
:1028A000CFE7FDF7B3FC0135164B5B5D002BC8D0BD
:1028B000605D5C2807D0012FF3D03368002BF2D085
:1028C000FDF798FCEFE72800FFF75AFF431C0AD0FA
:1028D0000335012F0DD043461B68002BE4D0C0B256
:1028E000FDF788FCE0E70A4A022311680B431360F6
:1028F000A7E7C0B2FDF78AFCD6E7C0464014002027
:1029000038140020C0130020A4140020101500204B
:0C291000A0140020B014002010020020D1
:10291C0030B5284B1B6880225202934228D3254B9A
:10292C00254A1A60254B1B88DB0711D4234B002248
:10293C001A821A802249CA6902200243CA61214ABA
:10294C001A83FA22D200DA621A8801210A431A8009
:10295C00184B1B68013B9BB2184A13851A4B1B681A
:10296C00002B22DB154A138C01210B4313841BE033
:10297C00002BD7D1114A13880124A3431380124B87
:10298C000121494219609023DB0518680F4D28403E
:10299C001860D9682940D960D86880218901014321
:1029AC00D960138CA343138430BD138C01218B434A
:1029BC001384F9E79C140020FFFF00000004004082
:1029CC00001002406060000080140020FFCFFFFF69
:1029DC009022D205136827490B401360264A138CAA
:1029EC0001218B431384254B1B68002B24DB902186
:1029FC00C905CA681F480240CA60002B24D0FA22BD
:102A0C00D20093422ADA9023DB05196880229201C6
:102A1C000A431A601A6A1A490A401A62196A802211
:102A2C0052040A431A62144B1A8C01210A431A8469
:102A3C00124A12685A6370479022D205D1688023DB
:102A4C009B010B43D360F6E70B000968802252010F
:102A5C000A431A608022D2039A61ECE7074B1A6092
:102A6C009023DB051968802252010A431A60402228
:102A7C009A61E0E7FFCFFFFF0004004080140020C4
:042A8C00FFFFFFF059
:102A9000324B9B6C002B60DD314A1268002A29DB27
:102AA00030490A60304A1268022A1ED008DC002A27
:102AB0000ED0012A45D19022D205022191610FE06A
:102AC000032A3ED19022D2058021890291613EE005
:102AD0009022D20580214902916180218902916171
:102AE00021490A6801320A6034E09022D2050121AE
:102AF0009161F5E752421B490A601B4A1268022A9B
:102B00001AD008DC002A0ED0012A1AD19022D20550
:102B100001219161E4E7032A13D19022D20580219B
:102B20004902916113E09022D2058021490291610E
:102B3000802189029161D3E79022D205022191611F
:102B4000CEE709490A6801320A60032A02DD064A13
:102B500000211160013B014A936470471008002076
:0C2B6000581400206C1400205C140020AD
:102B6C0010B5084B9B6C002B07D0074B1B68002B38
:102B7C0003DD064B1B68002B00D010BDFFF782FF56
:102B8C00FBE7C04610080020581400206C140020ED
:102B9C0010B50023064A1360064A1360064A1360F8
:102BAC00FFF7DEFFFFF7C6F80028F9D010BDC046CE
:0C2BBC004014002044140020A814002045
:102BC80010B5FFF7CFFF154B1B68022B17D0144B1E
:102BD8001868002817D0134B1B780020002B12D040
:102BE800FFF760FD00280ED0FFF7A6F801280BD0EC
:102BF80002280CD00C4B1868431E984103E0074B81
:102C080000221A60012010BDFFF78EFBF2E7064A8A
:102C180080235B0011680B431360EBE74814002026
:0C2C2800FC01002033150020A014002047
:102C340010B50D4B1B68012B05D00C4A40231168BD
:102C44000B43136010BDFEF783F8002804D1FFF78F
:102C5400B9FF0028F7D0F5E7054B1A68111D196074
:102C6400FF2318405060EDE710150020A014002049
:042C740070140020B8
:102C780010B5094A1368094918680860043B1360CD
:102C88000C002368002B05D0FDF7FCFBFFF798FF2D
:102C98000028F6D010BDC046701400209014002003
:102CA80010B5044B1A68642311684B431360FFF78F
:082CB800DFFF10BD70140020C5
:102CC000114A13681868043B136018280BD90300D5
:102CD000A03B182B05D90D4A8023DB0011680B435C
:102CE00013601F2318400300083B042B04D904235E
:102CF00002009A43122A05D1044A8023DB0011689E
:102D00000B4313607047C04670140020A0140020CD
:102D100010B5FFF7D5FF104B1B68002B0FD10F2804
:102D20000ED89023DB051B8A0122824013400B49F9
:102D30000A68101D0860002B0AD00123536010BDE3
:102D4000074B1B8A0F2210400E3A82401340EEE7D9
:102D500000235360F3E7C046A01400207014002045
:042D60000004004823
:102D6400062800D07047074B1B680133FAD0064A87
:102D7400138C01218B431384024B012252421A60AB
:0C2D8400F0E7C04680140020000400406E
:102D900070B5FFF795FF0400174B1B68002B14D18B
:102DA0000F2813D9400003228240144BD968914365
:102DB000D9601968914319601D6801221100814092
:102DC00029431960103CA2409A6170BDFFF7CAFF09
:102DD0006000032282409023DB05D9689143D960CB
:102DE0001968914319601D6801221100814029432F
:102DF0001960A2409A61E8E7A0140020000400488E
:102E000070B5FFF75DFF0400174B1B68002B13D153
:102E10000F2812D9400003228240144BD9689143F5
:102E2000D9601968914319601D6801221100814021
:102E300029431960A2409A6170BDFFF793FF6000BB
:102E4000032282409023DB05D9689143D960196839
:102E5000914319601D6801221100814029431960C6
:102E60001034A2409A61E7E7A01400200004004853
:102E700010B5FFF725FF0400144B1B68002B11D180
:102E80000F2810D9103C64000322A240104B19688F
:102E900091431960D9689143D960D9680122A24051
:102EA0000A43DA6010BDFFF75DFF64000322A24011
:102EB0009023DB05196891431960D9689143D96063
:102EC000D9680122A2400A43DA60EBE7A01400208F
:042ED00000040048B2
:102ED40010B5FFF7F3FE0400144B1B68002B10D150
:102EE4000F280FD944000322A240114B19689143C3
:102EF4001960D9689143D960D9680222A2400A4373
:102F0400DA6010BDFFF72CFF64000322A240902377
:102F1400DB05196891431960D9689143D960D96870
:102F24000222A2400A43DA60EBE7C046A014002064
:042F3400000400484D
:102F380010B5FFF7C1FE04000F4B1B68002B0BD127
:102F48000F280AD944000322A2400C4B1968914368
:102F58001960D9689143D96010BDFFF7FFFE64007E
:102F68000322A2409023DB05196891431960D968B0
:102F78009143D960F0E7C046A0140020000400483F
:102F880010B5144BDA6814490A40DA60996980224E
:102F980092000A439A61FDF79BF8FDF799F8FDF74F
:102FA80097F8FDF795F80D4B802212061A6100225A
:102FB800DA600B490A6004325A619A6801210A43AF
:102FC8009A60190001220B681A42FCD0FDF780F8BC
:102FD80010BDC04600100240FFFDFFFF0024014065
:042FE8000827014075
:102FEC000C4B1A6801210A431A609A6801310A4392
:102FFC009A60190001228B681A42FCD1064B9A691F
:10300C0006490A409A61D968802292000A43DA6024
:10301C007047C0460024014000100240FFFDFFFF36
:10302C00F0B589B004AA554B13CB13C21B8813807F
:10303C006A46534B13CB13C21B781370514B1B684E
:10304C001C68621C18D0072C03D92300A03B072B4B
:10305C001BD84D4B9B699B051ED54C4B4C4A1A609B
:10306C000F232340590003228A40072B00D97EE00E
:10307C009900484841588F46043B424A1360FFF779
:10308C00AFFF684603F0D7FD35E0434A8023DB00F1
:10309C0011680B4313602EE0FFF770FF04A803F0D8
:1030AC00CAFDDAE79021C905086810430860C868B2
:1030BC009043C86001229A401300344A936204265C
:1030CC00002714000425A3682B43A36023681D422A
:1030DC00FCD0236CFF18FCF7F9FF013E002EF2D157
:1030EC00284B1B68BA081A60BB0704D5254B1A6815
:1030FC0013680133136009B0F0BD9021C90508684D
:10310C0010430860C8689043C860D3E79021C90594
:10311C00086810430860C8689043C860CAE79021EB
:10312C00C905086810430860C8689043C860C1E7C7
:10313C001A490968013108D01948018C0124A143AE
:10314C00018416490120404208609021C905086895
:10315C0010430860C8689043C860ABE79021C9056C
:10316C00086810430860C8689043C860A2E70A4A20
:10317C008023DB0011680B431360BCE7EC6E000886
:10318C00FC6E000870140020001002400024014066
:10319C00FF070000C4630008A01400208014002066
:0431AC0000040040DB
:1031B0001A4B1B68032B25D8194B1B68043B1C2B8F
:1031C00020D880235B02174A12689A421AD2164B03
:1031D0001A6816490A401A6019688822D2000A4300
:1031E0001A60DA6812490A40DA60D96880229200CF
:1031F0000A43DA60094B1B68012B0AD90A4B0822E3
:103200009A6105E00B4A8023DB0011680B431360D1
:103210007047054B802212039A61F9E76014002081
:103220006814002064140020000400483FF0FFFFF1
:08323000FFFCFFFFA0140020C9
:1032380010B50A4A13680A4918680860191F11600E
:1032480008680849086019000839116008680649C3
:1032580008600C3B1360FFF7A7FF10BD7014002037
:0C32680064140020681400206014002092
:10327400F8B5DE4657464E464546E0B5B54B1B68A5
:10328400A822D2001340013AFF3A93421BD1B24B19
:103294001B681C68B14B1A68B14B186800286DD1C3
:1032A400AC4B802109039961AE4B1B68002B0DD1F7
:1032B4000125A84880218903884620218C4680273F
:1032C4003F03082644E0FFF771FFE0E701239B4634
:1032D400A04D80239B039A462023994680231B03F9
:1032E4009846A04B9C46A0491F001EE05346AB6184
:1032F4004346AB6163461B68002B04D09B4E316090
:10330400013B002BFBD140002B8A1B095E46334056
:1033140018430823AB613B68002B04D0934E316003
:10332400013B002BFBD1002A1BD0013A5B469340A2
:103334001C42DBD04B46AB61DAE7414681618761D1
:103344005900038A1B092B400B438661002A07D0CE
:10335400013A290091400C42EFD061468161EEE7C9
:1033640018007C4B802212039A617B4B1B68186007
:10337400F0BCBB46B246A946A046F8BD012814D00D
:10338400022875D0734B08219961764B1868002880
:1033940000D0CDE001256F4980239B03984620236C
:1033A4009C4680273F03082614E16A4B80210903C9
:1033B40099616C4B186800280AD10125654980235E
:1033C4009B03984620239C4608278026360342E028
:1033D400002001239B465F4D80239B039A462023B4
:1033E4009946183B98465F4B9C465F491F001FE077
:1033F4005346AB614346AB6163461B68002B04D064
:103404005A4E3160013B002BFBD140002B8A1B0933
:103414005E463340184380231B03AB613B68002B9B
:1034240004D0524E3160013B002BFBD1002A1AD04C
:10343400013A5B4693401C42DAD04B46AB61D9E774
:1034440043468B618F6140000B8A1B092B40184354
:103454008E61002A07D0013A2B0093401C42EFD022
:1034640063468B61EEE73B4B802212039A617CE753
:10347400384B082199613B4B186800280AD1012573
:10348400344B80218903884620218C4608278026D6
:10349400360341E0002001239B462E4D80239B03ED
:1034A4009A4620239946183B98462E4B9C462E4913
:1034B4001F001FE05346AB614346AB6163461B6884
:1034C400002B04D0294E3160013B002BFBD140007E
:1034D4002B8A1B095E463340184380231B03AB61D0
:1034E4003B68002B04D0214E3160013B002BFBD103
:1034F400002A19D0013A5B4693401C42DAD04B466D
:10350400AB61D9E7414699619F614000198A29401E
:1035140008439E61002A07D0013A290091400C42D9
:10352400F0D061469961EFE70A4B08229A611CE7E3
:10353400002001239B46074D80239B039A462023AA
:10354400994680231B039846064B9C4606491F0058
:103554002DE0C046000400487014002068140020C8
:103564006014002064140020AAAA00000030004067
:103574005346AB614346AB6163461B68002B04D0E2
:103584001A4E3160013B002BFBD140002B8A1B09F2
:103594005E46334018430823AB613B68002B04D0DC
:1035A400124E3160013B002BFBD1002A1AD0013AA4
:1035B4005B4693401C42DBD04B46AB61DAE74346A3
:1035C4008B618F6140000B8A1B092B4018438E616D
:1035D400002A07D0013A2B0093401C42EFD06346E7
:1035E4008B61EEE7024B08229A61BEE60030004090
:0435F4000004004887
:1035F80010B5074A1368191D1160064A12685A6007
:10360800FF20FEF745FEFF20FEF742FE10BDC04634
:0836180070140020B014002022
:10362000F8B5104E33681D6801350F4C2D19280A66
:10363000FF273840FEF730FE38002840FEF72CFE0A
:103640000A4B1B68013B1B193268190A1068215488
:103650001268A41863707620FEF71EFE3368043BE0
:103660003360F8BD7014002010020020B014002058
:1036700070B57E280DD8C0000E4D441908352D18A0
:103680002078002804D0FCF7C1FD0134AC42F7D10A
:1036900070BD7F2528400001074D441908352D18BD
:1036A00020780028F4D0FCF7B1FD0134AC42F7D10A
:0C36B000EEE7C04620670008100800206C
:1036BC0070B50001064D441908352D1820780028E6
:1036CC0004D0FCF79DFD0134AC42F7D170BDC0466F
:0436DC0010080020B2
:1036E000F0B5C64600B582B0A34B1A6800929B881D
:1036F0006A469380A14B1D68002D03D002B080BCA8
:10370000B846F0BD9E4B1B689E4A13601B789846D6
:103710001F009D4B1B685E00F6180D20FCF776FD20
:10372000002E06D02C002020FCF770FD0134A642AC
:10373000F9D1944B188803F09AFC2020FCF766FD21
:10374000404603F094FC2020FCF760FD7F2F1AD840
:103750004046FFF78DFF6B2F53D06C2F57D06D2F46
:1037600000D182E06E2F00D187E06F2F56D0712FED
:1037700000D18AE0722F00D18DE0FD224346733BD9
:1037800013424BD059E02D20FCF740FD3E20FCF7C2
:103790003DFD2020FCF73AFD4046FFF769FF784BDE
:1037A0001B685B787F241C40692F00D19EE06A2F44
:1037B00000D1A5E0642F00D1B7E0744C032D00D1F7
:1037C000C7E02368022B00D8C3E0FCF75FFEFEF7DA
:1037D0006DFF0028F2D0FEF7B3FA0500012800D1F2
:1037E000ADE0022800D1ADE00428E7D1664B1B68AC
:1037F000002B00D1ADE0664A1360644B02221A60D0
:10380000DCE7644B1B681B68002B07D0C7E7614BE4
:103810001B68191F1A680B689A42C0D0684603F0EB
:1038200010FA574B1B68587800029B7818430130F8
:1038300003F01DFC2920FCF7E9FC682F35D1504B23
:103840001B685C782820FCF7E1FC534B1B68102BAD
:1038500027D02000FDF79AF82920FCF7D7FC484B29
:103860001B685B787F241C40A1E74A4B1B681A1F2A
:1038700012681B689A42D1D291E7464B1B681A1F07
:1038800012681B689A42C9D989E7424B1B681B68BA
:10389000002BC3D083E73F4B1B681B68002BBDD1B7
:1038A0007DE7200003F0E3FBD6E7672F00D076E743
:1038B000334B1A6893781B04517809060B4311792E
:1038C0000B43D47824021C432820FCF79FFC324B86
:1038D0001B68102B06D02000FDF758F82920FCF7B4
:1038E00095FC67E7200003F0C2FBF7E72820FCF710
:1038F0008DFC2000FFF7E2FE2920FCF787FC5CE747
:103900002820FCF783FC2000FFF7D8FE4020FCF7BE
:103910007DFC20010830214C00190004000C03F04C
:10392000DCFB2920FCF772FC47E72020FCF76EFC4B
:103930003C20FCF76BFC2D20FCF768FC3DE7FEF714
:10394000F7FC3BE70D4A80235B0011680B431360D3
:10395000D4E62020FCF75AFC43465F3B022B03D8F9
:10396000684603F06EF9C9E67B20FCF74FFC202087
:10397000FCF74CFCC2E6C0463C6C0008A0140020DA
:1039800098140020941400208C140020FC010020C6
:10399000BC140020701400205014002010080020D7
:1039A00010B5FFF79DFE074B1B68002B08D1064B97
:1039B0001B681B789B00054A9B589847FEF706FE3C
:1039C00010BDC046A0140020981400200000002064
:1039D00010B51B4A1368013313601A4B1A68111D86
:1039E000196019490B6853601A787F2313401B0133
:1039F000164AD3189B680B601B787E2B0BD8144A91
:103A00001268032A04D09B00124A9B58984710BDA5
:103A1000FFF7C6FFFBE70E4B1B68032B06D00E4BD0
:103A20001B68002BF3D1FFF7D3FFF0E7FFF758FE39
:103A3000094B1B68002BEAD1FEF7C8FDEFE7C04633
:103A40008C14002078140020981400201008002006
:0C3A5000FC01002000000020A014002059
:103A5C00F0B587B001AA3D4B13CB13C211001A6805
:103A6C000A601B790B713A4C3A4BE4183A4B1B68C1
:103A7C00A34265D2394D384E2F003DE0FDF762FF71
:103A8C0041E0FFF79FFF28E0FEF70AFE00280CD16B
:103A9C0033681B787E2B1BD8304A1268032A14D04B
:103AAC009B002F4A9B58984717E0FEF743F90128D3
:103ABC0008D00228ECD12B4A80235B0011680B4301
:103ACC0013603DE0FEF72EFCE2E7FFF763FF04E036
:103ADC003B68032B21D0FFF775FFFFF741F8214B13
:103AEC001B68002B2CD11C4B1B68002B1AD00133EC
:103AFC00194A1360A34223D22B68002BC4D11A4B52
:103B0C001B68042BBAD0144B1B681B787E2BB8D8BF
:103B1C009B00134A9B589847DFE7FFF7DBFDFEF746
:103B2C004FFDD8E70D4B1B68032B0BD00B4B012221
:103B3C001A6000230D4A13700D4A13600D4A13606E
:103B4C0007B0F0BD01A803F076F8EFE7186F000896
:103B5C0010020020000E002098140020FC01002010
:103B6C0000000020A0140020481400203315002071
:083B7C00B81400208C14002095
:103B8400F8B5274B1C68002C2ED1264B1B68190155
:103B9400254A5218D168C022120511420AD0234A7C
:103BA4001168081D10601B011F4AD3189B684B60E5
:103BB4002000F8BD1B011C4AD3189A681C4B1A60DC
:103BC4001C4B01221A701C4D2F681C4C2668522372
:103BD4002B6023601A4B00221A60FFF73DFF2F6011
:103BE4002660184B1C68E3E70E4B186802010E4B65
:103BF4009B18DA68C0231B0514001C401A4204D128
:103C040080231843FEF746FBD2E76920FEF742FB08
:103C1400044B1868FEF73EFB0A4B1C68C8E7C04615
:103C2400A41400207C14002010080020701400202C
:103C34009814002033150020441400204014002060
:083C4400A8140020A0140020C8
:103C4C0070B50023384A1370384A1360384A136031
:103C5C001500384E0EE0384B1B68FF2B24D868201B
:103C6C00FEF714FB344B1868FEF710FB304B1A6848
:103C7C002E4B1A60314C2B682268934230D2FEF7DF
:103C8C0051F93378002BF6D0FEF7ECF900281FD051
:103C9C002B4B1B68002BDED12A4A1368191D1160AF
:103CAC00254A12685A60E1E76720FEF7EFFA224CCA
:103CBC0003202056FEF7EAFA0223E05EFEF7E6FA4E
:103CCC0023681812FEF7E2FA2068FEF7DFFACDE758
:103CDC00FEF772FA002809D0FFF74EFF002800D03B
:103CEC0070BD134B1A68114B1A60C3E7FEF728FA24
:103CFC0000280AD0FEF7E2FA134B1B68002BEFD119
:103D0C000B4B1A68094B1A60B4E70F4A0123116870
:103D1C000B4313600D4B1A680D4B1A60044B1A6859
:103D2C00024B1A60DCE7C046331500203814002023
:103D3C0040140020C01300203C1400204414002028
:103D4C00A414002070140020A0140020AC14002037
:043D5C00B01400207F
:103D6000F0B5DE4657464E464546E0B591B00BA944
:103D7000B94B0A0013CB13C203CB03C206AAB74B3D
:103D800013CB13C211001A680A609A888A809B7943
:103D90008B7102AAB24B13CB13C21B881380B14B99
:103DA0001A68B14B1A60FEF7C3F8FEF70BFA002849
:103DB0000DD1FEF7CBF9002805D1AC4A01231168DB
:103DC0000B43136018E10BA802F03BFF14E1A54B75
:103DD0001A68A54B1A6006A802F033FFA44D2B68A1
:103DE0001801A44C001903F078F90D20FCF70EFA25
:103DF0002B681A01A418E168C022120508001040BF
:103E00000190114200D0FEE01B019A4AD3189C6831
:103E1000994BE41A2405240D1B5D0125642B00D168
:103E2000D1E0954E24E00D20FCF7F0F9019D1FE054
:103E3000914B1A195078000202341F5D0743282065
:103E4000FCF7E4F9781C03F012F92920FCF7DEF9FD
:103E500001352020FCF7DAF92020FCF7D7F90134EE
:103E6000854B1B5D642B00D1ADE00135072DDAD801
:103E7000A0190004000C03F0FAF83A20FCF7C6F988
:103E8000305DFFF7F5FB335D1A006B3A0A2ACFD994
:103E9000682B1AD0672B2ED0692B4CD06A2B57D0A9
:103EA000652BD6D12220FCF7B1F9734B1B195B7837
:103EB0009B46A31C98465B46002B7DD06E4B43442B
:103EC00099465C460F239A466BE001342820FCF7A4
:103ED0009DF96A4B1B68102B08D0674B185DFCF7E7
:103EE00055FD2920FCF792F90135B2E7624B185DC8
:103EF00003F0F3F8F5E76048021993781B04517852
:103F000009060B43D7783F020434025D13431F4375
:103F10002820FCF77BF9594B1B68102B07D0380081
:103F2000FCF734FD2920FCF771F9013591E73800E1
:103F300003F0D3F8F6E701342820FCF767F94E4B7D
:103F4000185DFFF7BBFB2920FCF760F9013580E71E
:103F500001342820FCF75AF9474B1F5D3800FFF762
:103F6000ADFB3F01083743483F184020FCF74EF9AE
:103F70003804000C03F0B1F82920FCF747F90135AB
:103F800067E75C20FCF742F9380902F04CFE504626
:103F9000384002F048FE013C01239C46E144002CDD
:103FA00009D04B461F783B00203B5E2BE9D83800F8
:103FB000FCF72CF9EFE7D8444446013C2220FCF7FB
:103FC00025F9033545E72C4820180004000C03F0C0
:103FD0004EF83A20FCF71AF93B20FCF717F9244B6E
:103FE0001A681201234B9B18DA68C0231B051A427A
:103FF00009D10D20FCF70AF911B0F0BCBB46B2465E
:10400000A946A046F0BD02A802F01BFE1B4B1B6890
:10401000102B18D0164B1A681201164B9B18986873
:1040200002F0BDFE2020FCF7F1F84020FCF7EEF88E
:104030000F4B1868000108300E4BC0180004000C2C
:1040400003F04BF8D5E70A4B1A681201094B9B188D
:10405000986803F042F8E5E75C6C0008706C0008B3
:10406000846C00084014002038140020A0140020A4
:104070007C140020100800201002002050140020A2
:10408000134B1B68134A1360134A12681201134939
:104090005218BE20C000844661448A420AD21049A8
:1040A0000139891A8908013189005118002001C29B
:1040B0008A42FCD10B4A934209D80B4A9B180B4900
:1040C0008C4662440021197001339342FBD1704742
:1040D000B0140020AC140020881400201008002028
:1040E000000E0020FE05000010020020FF05000069
:1040F00010B5164B1A68164B1A60FDF719FFFEF73C
:1041000061F800280DD0114B1A68114B1A60114B41
:104110001B68042B0BD8104A802311680B431360D3
:1041200004E00D4A212311680B43136010BD0B4AB4
:1041300013600B4A1B0100219954D318DB681B053F
:104140001B0D084A1360FFF79BFFEFE740140020A8
:10415000381400207C140020A014002088140020B3
:0841600010080020B01400203B
:1041680010B50023204A1360204A1360204A1370B8
:10417800204A1360204A1360204A01211160204A16
:104188001360204B1A68204B1A60204A00231178CC
:10419800002903D0013310325F2BF8D11C4A136079
:1041A8001C4A1D4BD35C642B1CD01B4B1100013BDC
:1041B800CA5C642A02D0002BF9D102E0002B00D09F
:1041C8000133164A1360FFF757FF154A154B1A605B
:1041D80000231360144A0F491160144A1360FDF755
:1041E8000BFA10BD0C4BEBE7A8140020A414002018
:1041F80033150020B81400208C140020FC01002086
:104208004C140020841400205014002010080020B2
:104218008814002010020020FF050000B0140020C0
:10422800F81200207814002098140020A014002010
:1042380030B5B9B036AAA04B1968369199889180E3
:104248009B79937134AA9D4B196834919988918010
:104258009B79937131AA9A4B03CB03C211001A8838
:104268000A809B788B702EAA964B13CB13C22BAA6D
:10427800954B03CB03C211001A880A809B788B7078
:1042880027AA924B13CB13C21B88138022A9904BE9
:104298000A0013CB13C203CB03C21CA98D4B0A001F
:1042A80013CB13C203CB03C21B78137018AA8A4B13
:1042B80013CB13C21B68136014AA884B13CB13C209
:1042C8001B8813800FAA864B13CB13C211001A68E0
:1042D8000A609B888B8009A9824B0A0013CB13C202
:1042E80003CB03C21B78137005AA7F4B13CB13C2F1
:1042F8001B78137001AA7D4B13CB13C21B88138044
:104308007B4B1A687B4B54339A4200D280E07A493F
:104318000423086803430B60764B0C339A4204D29B
:10432800754A042311680B431360744B1B68002BF8
:104338000FD0734B1968734B09010022CA545B18DC
:104348005A709A70DA701A715A719A71DA719A60A1
:10435800DA606A4B00221A606B4B1B68002B0ED088
:104368000024694D2020FBF74DFF01342B68A34240
:10437800F8D85E20FBF746FF0D20FBF743FF36A871
:1043880002F05BFC5C4C206802F06DFE3D20FBF700
:1043980039FF2368DB075ED4574B1B689B075ED445
:1043A800554B1B685B075ED4534B1B681B075ED4D9
:1043B800514B1B685B065ED44F4B1B689B065ED453
:1043C8004D4B1B681B065ED44B4B1B68DB055ED44C
:1043D800494B1B689B055ED4474B1B685B055ED445
:1043E800454B1B681B055ED434A802F026FC464BDF
:1043F8001868FCF7C7FA2920FBF704FFFFF7B0FE9F
:104408000D20FBF7FFFE414B00221A6039B030BD8A
:10441800384B0C339A4200D282E7374B1B68002B8B
:1044280000D082E7354B1B68002B40D1384B1B6806
:10443800012BE5D02020FBF7E5FE6F20FBF7E2FE1D
:104448006B20FBF7DFFE334B1B68102BD8D14820BD
:10445800FBF7D8FED4E731A802F0EFFB9CE72EA8C3
:1044680002F0EBFB9CE72BA802F0E7FB9CE727A8F0
:1044780002F0E3FB9CE722A802F0DFFB9CE71CA804
:1044880002F0DBFB9CE718A802F0D7FB9CE70FA81B
:1044980002F0D3FB9CE714A802F0CFFB9CE709A825
:1044A80002F0CBFB9CE705A802F0C7FB9CE701A83C
:1044B80002F0C3FBA4E7C046C46C0008CC6C00083B
:1044C800D46C0008E06C0008EC6C0008F86C00087C
:1044D800086D00081C6D0008346D0008446D000864
:1044E800546D0008686D0008806D0008906D000824
:1044F800701400205C130020A0140020A4140020D5
:10450800881400201008002038140020B814002057
:08451800A8140020501400203B
:1045200010B50023244A13600A2224490A60244952
:104530000A60244A01211160234A1360234A136050
:10454000234A07311160234A2A311160224A13603D
:10455000224B012252421A60214B32325624002152
:10456000C02000051C705A709970D8609960103393
:104570000132D2B2352AF5D1194B0B324E21995462
:104580000132053199540132013199540439013213
:104590009954002244201A54C0200005D8640120F8
:1045A000404298640F48052404605A540E4B1A6028
:1045B000FFF7DAFD10BDC046181500208414002056
:1045C00050140020FC010020C014002060140020C2
:1045D00068140020641400209C1400208014002023
:0C45E0001008002088140020B0140020F7
:1045EC0070B5164C164D2B682360FDF79BFC2B68A1
:1045FC002360144B1D68013D28006B1C17D02D0146
:10460C00114BED18114E10E08B420BD1002913D039
:10461C000132A95C935D1C00613C192CF4D8203B41
:10462C00DBB2F1E7103D013804D30022F1E70120A1
:10463C00404201E00120404270BDC04638140020C9
:10464C00401400208814002010080020C013002003
:10465C0010B5FFF7C5FF0400431C0DD002011D4B24
:10466C009B18DA68C0231B051A420BD01A4A802308
:10467C0011680B43136010BD174A212311680B43BB
:10468C001360F8E7FFF7ACFF431C11D00201114B8C
:10469C009B18DA68C0231B051A420FD1844213D928
:1046AC000C4B24011C19A268000118188260E2E767
:1046BC00094A212311680B431360DCE7064A802367
:1046CC0011680B431360D6E7034A802311680B4330
:0C46DC001360D0E710080020A01400209C
:1046E80010B5FFF77FFF431C0FD003010D4AD21806
:1046F800D3681B051B0D0C495B1892689A420AD3B4
:104708000001084A1018836010BD084A2123116867
:104718000B431360F8E7054A802311680B431360C5
:10472800F2E7C0461008002010020020A014002064
:10473800F8B506000D490A68571C0F6054783F19F0
:10474800002C10D00D0005E05878FBF75BFD013C0C
:10475800002C08D02B685A1C2A60012EF4D05878F7
:10476800FBF744FDF3E7014B1F60F8BD98140020E8
:10477800074B1A68511C196051780902901C18607F
:1047880092781143802292050A431A607047C04606
:044798009814002051
:10479C0010B5084B1B681B68002B08D0064A136821
:1047AC0002331360034A1368043B136010BDFFF718
:0C47BC00DDFFF7E77014002098140020C7
:1047C80010B5094B1B68191F1A680B689A4208D163
:1047D800064A136802331360034A1368043B1360E4
:1047E80010BDFFF7C5FFF7E77014002098140020EC
:1047F80010B5094B1B68191F1A680B689A4208DD27
:10480800064A136802331360034A1368043B1360B3
:1048180010BDFFF7ADFFF7E77014002098140020D3
:1048280010B5094B1B68191F1A680B689A4208DAF9
:10483800064A136802331360034A1368043B136083
:1048480010BDFFF795FFF7E77014002098140020BB
:1048580010B584B001A8214B020012CB12C21B88EC
:10486800138002F0EAF91E4C2068FCF78BF82368E5
:104878001F2B15D00B2B1DD0194B1B68132B20D0C9
:10488800174B1B68262B20D0154B1B68392B20D0C3
:104898003020FBF7B7FC3020FBF7B4FC04B010BDA8
:1048A8003220FBF7AFFC3520FBF7ACFC3020FBF7E0
:1048B800A9FCF3E73520FBF7A5FC3220FBF7A2FCA7
:1048C800DAE73220FBF79EFCDAE73420FBF79AFCA4
:1048D800DAE73620FBF796FCDAE7C046AC6D00084D
:0448E800281500206F
:1048EC0070B5AEB0C34B1A682C929A886946B42046
:1048FC0009180A809B796A46B621521813702AADA2
:10490C00BD4B2A0003CB03C2BC4B1A6828929A8871
:10491C006946A42009180A809B796A46A621521878
:10492C00137024ACB64B220043CB43C21B781370DC
:10493C00B44B1A6822929A8822AB9A80B24B1A68AE
:10494C0020929A8820AB9A801CAAB04B43CB43C2CE
:10495C001B68136019AAAE4B43CB43C214AAAD4BD0
:10496C0043CB43C211001A680A601B790B71AA4B26
:10497C001A6812921A7912AB1A710EAAA74B43CB72
:10498C0043C21B8813800BAAA54B03CB03C21B7815
:10499C001370A44B0A9308AAA34B03CB03C2A34BDB
:1049AC001A6806929A8806AB9A8003AAA04B03CB8E
:1049BC0003C21B78137001AA9E4B03CB03C2442085
:1049CC00FBF71EFC6120FBF71BFC7420FBF718FCAB
:1049DC006120FBF715FC2CA802F02DF996480C3041
:1049EC0002F03FFB280002F026F92CA802F023F974
:1049FC00924802F036FB200002F01DF9904802F0BC
:104A0C0030FB28A802F017F98E4802F02AFB0D2083
:104A1C00FBF7F6FB8C4B1B68002B10D122A802F085
:104A2C000AF91CA802F007F919A802F004F9874B3F
:104A3C001B680024002B06D0824E844D6AE020A80F
:104A4C0002F0F9F8EDE76E20FBF7DAFB6F20FBF7CD
:104A5C00D7FB6E20FBF7D4FB6520FBF7D1FB0D20B9
:104A6C00FBF7CEFBFFF7F2FE794B1B680222934358
:104A7C00012B02D014A802F0DEF80D20FBF7C0FBCE
:104A8C0012A802F0D8F8734B1868FBF779FF2C20AA
:104A9C00FBF7B6FB704B1B68102B43D06F4B1868A1
:104AAC00FBF76EFF2C20FBF7ABFB6D4B1868FBF78D
:104ABC0067FF0EA802F0BFF86A4B1E68002E3DD1AE
:104ACC000020FBF75DFF0BA802F0B5F8664B1868E9
:104ADC00002800DA73E0604B1B68102B00D172E0E9
:104AEC00FBF74EFF08A802F0A6F8564B9B6C01335F
:104AFC0000D06FE09023DB059B8ADB0766D401A80E
:104B0C0002F099F80D20FBF77BFB2EB070BDFBF784
:104B1C0077FB01342B68013B1B01F318185D00284F
:104B2C00F5D19CE74D4B186802F0D1FA2C20FBF71D
:104B3C0067FB4B4B186802F0CAFABAE77501AD1B5C
:104B4C00AD00AD192D012900484802F0EAFA040025
:104B5C00FBF716FF6643B404A41BA400A41BE400DB
:104B6C00A4192401A41B6401414B9C4664442E20CF
:104B7C00FBF746FB2900200002F0D3FAFBF700FFFD
:104B8C002900200002F058FA8C00641864002900F7
:104B9C00200002F0C6FA06002900200002F04CFAB0
:104BAC00880040184000290002F0BBFA042383421D
:104BBC009B415B42F6183000FBF7E2FE83E70AA844
:104BCC0002F039F88EE702F082FA8BE72D20FBF722
:104BDC0017FB94E706A802F02EF8264B1868FBF793
:104BEC00CFFE03A802F027F8164B986CFBF7C8FE13
:104BFC0088E7C046E4630008EC630008F46300082F
:104C0C00FC6300080C640008146400081C640008B1
:104C1C002C640008386400084C64000854640008D4
:104C2C00646400084F46460070640008786400080D
:104C3C00806400088C6400085C130020F8120020CB
:104C4C00100200201008002018150020C0140020AD
:104C5C00101500206014002050140020681400204F
:104C6C00641400209C14002080140020006CDC02D2
:084C7C0000389C1C58140020B4
:104C840030B58BB003A8124B020032CB32C232CB08
:104C940032C21B8813806A460E4B32CB32C201F0FB
:104CA400CEFFFCF781F80028FBD0FF2318405928D9
:104CB40008D0684601F0C3FF0D20FBF7A5FA0020D9
:104CC4000BB030BD0D20FBF79FFA0120F8E7C0467A
:084CD40094640008B0640008BC
:104CDC00F0B591B0040001A9334B0A0023CB23C2D9
:104CEC0023CB23C223CB23C203CB03C22F4D304E85
:104CFC0033682B60FDF716F933682B60FDF7B2F9BA
:104D0C00051E08D02B4A802311680B431360002525
:104D1C00280011B0F0BDFDF713FA002804D10CA83F
:104D2C0001002A00244F0EE001A801F084FFFFF7D8
:104D3C00A3FF0028F3D10225EAE7002B12D0072AA3
:104D4C000AD001320131D35D0B701E00613E192E69
:104D5C00F3D8203B0B70F2E7164A022311680B4381
:104D6C001360D5E70CAB1B78002B0CD0134A1268E0
:104D7C00120113495218535501354378002B02D0B8
:104D8C000130072DF7D10D4B1A6812010C4B9B18F3
:104D9C005D1900226A700B4A10680B4A82189A60DF
:104DAC002043D8600125B3E7BC6400083814002008
:104DBC0040140020A0140020C013002088140020F0
:0C4DCC0010080020B0140020100200208D
:104DD80070B5C0200005FFF77DFF00280DD00A4CF4
:104DE80022680A4803681D010949491915688D6038
:104DF800043A22600133036070BD064A012311683A
:104E08000B431360F8E7C046701400208814002094
:084E180010080020A014002086
:104E200010B50020FFF75AFF002808D0022807D04D
:104E3000074B1A68074B1A60074B01221A6010BD16
:104E4000064B1B681B01064A00219954F7E7C04630
:104E5000B0140020AC140020A414002088140020FA
:044E60001008002016
:104E640010B584B06A461F4B13CB13C21B88138042
:104E74001D4A13681C68043B1360962C1BD0112C2C
:104E840026D0192C03D113240B2C18D002E0312C7A
:104E940012D11F24132C12D01F2C10D0262C0ED06C
:104EA400392C0CD0602C0AD0104A8023DB00116806
:104EB4000B4313600AE06024382C0AD12624684688
:104EC40001F0BDFEFFF7DCFE002806D104B010BDE2
:104ED4000B24572CD8D13924F1E7054B1C60FBF780
:104EE40005F9F3E7EC6D000870140020A01400200D
:044EF400281500205D
:104EF80010B588B001A91B4B0A0013CB13C213CB02
:104F080013C21B881380184A13681C68043B13607B
:104F1800164B1B68A34208D0154B1B68002B06D004
:104F2800012C0DD813D0114B1C6008B010BD114ACC
:104F3800803311680B4313600C4B00221A60F4E7AE
:104F48000C4A8023DB0011680B431360EDE701A8CE
:104F580001F073FE0D20FBF755F9FFF78FFE0028CF
:104F6800E1D1E2E7046E000870140020101500205B
:084F78002C140020A0140020FD
:104F800030B585B0174B1A6802929A8869468A81B3
:104F90009B798B73144B1A6800929A888A809B794C
:104FA0008B71FBF7D3FF114C23681D6802A801F039
:104FB00048FEFCF73BFD2020FBF728F923681C681E
:104FC000684601F03EFEFCF731FD2020FBF71EF99C
:104FD000FFF758FE002803D0054B1D60054B1C60F1
:104FE00005B030BDE86F0008F06F000870140020B5
:084FF000C41400201C15002070
:104FF80030B589B001A80B4B020032CB32C232CB9C
:1050080032C21B68136001F018FEFFF737FE002854
:1050180001D109B030BDFBF7A5FA034B01221A6094
:0C502800F7E7C046E864000818150020F7
:1050340010B58CB006A91E4B0A0013CB13C203CBC8
:1050440003C21B78137069461A4B0A0013CB13C2B0
:1050540003CB03C21B781370174A13681968043B07
:10506400136001290ED8002914D1684601F0E7FD28
:10507400FFF706FE00280BD0104B00221A60FFF742
:105084004DFA05E00E4A8023DB0011680B431360E0
:105094000CB010BD06A801F0D2FDFFF7F1FD002809
:1050A400F6D0064B01221A600120FBF7C3F8EFE7A4
:1050B400386F0008506F0008701400201815002085
:0450C400A014002014
:1050C800074B1B68002B09D0054B00221A60054AC4
:1050D8001368191D1160044A12685A607047C04667
:0C50E800B814002070140020B414002044
:1050F40010B5214B1A68214B1A60FCF717FFFDF716
:105104005FF8002821D01C4B1A681C4B1A601C4BFA
:105114001A6812011B4B9B18DA68C0231B051A423C
:1051240019D0194B1B78002B1BD1184B1B68002B73
:105134001AD117480368124A11680901114A521812
:1051440019689160043B036004E0124AA0231168CB
:105154000B43136010BD0F4A802311680B43136087
:10516400F8E7FFF7AFFFE0E76A20FDF793F8044B99
:105174001868FDF78FF8EDE740140020381400207C
:105184007C1400201008002033150020A4140020F3
:0851940070140020A01400209B
:10519C0010B5094B1B78002B0BD1084A1368084932
:1051AC0018680860043B1360FDF7B2FBFDF710FCB8
:1051BC0010BDFFF783FFF0E73315002070140020BB
:0451CC009C1400200F
:1051D00010B50D4B1B78002B0DD10C4A13680C49F0
:1051E00018680860043B13600A4B1B88DB0705D571
:1051F000FDF7F4FB10BDFFF767FFEEE7064B182243
:105200001A60FDF78BFBF3E73315002070140020C4
:0C52100080140020000400409C140020CA
:10521C0010B5344B1B78002B2FD1334B9B6C0133C7
:10522C002ED0324B1B68002B0DD1314A1360314A02
:10523C0013609023DB051A680F218A431A601A68E1
:10524C000A390A431A602C490B681A68274802600D
:10525C00043B0B60002A0AD19023DB05802252020A
:10526C009A61802292029A611F4B00229A64214B10
:10527C0000221A60FDF706FC10BDFFF71FFFCCE7FC
:10528C001A4B00221A609023DB051A680F218A43FF
:10529C001A601A680A390A431A60174B1A6813689D
:1052AC00002B09DD9023DB05802252029A61022239
:1052BC009A61FFF787FFDFE7002B08DB9023DB0504
:1052CC00802252029A61802292029A61F1E75B423B
:1052DC0013609023DB0501229A61802292029A616D
:1052EC00E7E7C046331500201008002058140020B2
:0C52FC005C1400206C14002070140020D2
:10530800F0B5C64600B588B069462B4B0A0013CBEA
:1053180013C213CB13C203CB03C2284B1B78002B39
:1053280014D1274A13688024A40519680C43043B48
:105338001360244B9C420CD9234A8023DB0011685C
:105348000B43136008B080BCB846F0BDFFF7B8FE49
:10535800E7E70D20FAF756FF684601F06EFC2000DB
:1053680001F081FE270080370F25032398460FE0C0
:105378000D20FAF747FF200001F075FE3A20FAF7F2
:1053880041FF300001F081FC00250134BC420ED001
:1053980026780135102DEBD0300001F076FC43461D
:1053A8002B40032BF1D17C20FAF72CFFEDE70D20E1
:1053B800FAF728FFC6E7C046046500083315002041
:0C53C80070140020807F0020A014002042
:1053D40082B03A4B1A6801210A431A605A68384865
:1053E40002405A601A68374802401A601A68364800
:1053F40002401A605A68354802405A60DA6A0F203F
:105404008243DA621A6B324802401A635A6B8A4347
:105414005A6300229A600092019219688022520213
:105424000A431A60190080229202A020C0010B686E
:1054340013400193009B01330093019B002B02D185
:10544400009B8342F3D11D4B1B689B0306D50123AC
:105454000193019B012B04D002B0704700230193F8
:10546400F7E71C4B11221A60144B5A685A605A68A9
:105474005A605A6818490A405A6059688822520387
:105484000A435A601968802252040A431A601900B8
:10549400802292040B681342FCD0084B5A68032103
:1054A4008A435A605A6801390A435A6019000C2227
:1054B4004B681340082BFBD1CEE7C04600100240D6
:1054C4000CB8FFF8FFFFF6FEFFFFFBFFFFFFC0FF76
:0C54D400ACFEFFFF00200240FF7FC0FF85
:1054E0004C4B80221A6000224B4B1A604B490868D3
:1054F00080231B0203430B60494B1A601B68494A17
:105500009A1849490A6049490A604949581849495D
:105510000860494958184949086049495818494993
:105520000860494958184949086049495818494983
:105530000860494958184949086049498C466344FC
:1055400048490B60484B1B68002B06D113001833E9
:1055500046490B60464902330B6040231380354BAC
:105560001B6800221A80354B1B6880211980354B3F
:105570001B6840491980354B1B688020400018800B
:10558000344B1B681A80284B1B689881DA810130E4
:10559000FF3018825A82314B1B681880314B1B68D0
:1055A0001980314B1B68002B0BD1304B1B68C0217D
:1055B000890019802E4B1B681A801B4B1B6899832E
:1055C000DA832D4B2D4A1A802D4B2E4A1A802E4BF2
:1055D0002E4A1A80244B1B68002B02D12C4B2D4ADB
:1055E0001A802D4BBF2212021A6000232B4A13602F
:1055F0002B4A13602B4A2C490A602C490A602C4A1A
:105600002C490A602C490A602C4A13702C4A1370EA
:105610007047C0464C5C004034140020585C004089
:10562000505C00400060004030140020FC1400205A
:1056300002600040E81400200460004000150020D3
:1056400006600040EC14002008600040F8140020C0
:105650000A600040E414002014600040F4140020AC
:1056600016600040E014002028140020F0140020F0
:10567000DC1400200084FFFF005C004020320000AA
:10568000045C004031300000085C00403230000013
:105690000C5C004033360000405C004014140020D5
:1056A0002C140020000E0020D0140020CC14002068
:1056B000CC110020D8140020D414002001110020A7
:0456C0009112002023
:1056C40070B5204CE36980252D042B43E361FAF780
:1056D40001FD23691D432561FAF7FCFC236B80223D
:1056E400134323632369184A134023619022D2058C
:1056F400136816490B401360154B0021154A198095
:1057040002339342FBD1144B0021144A1980023313
:105714009342FBD1124A116880231B020B4313608E
:10572400104C01232360C820FAF710FF00232360E4
:10573400094A1360FFF7D2FE0B4B802212061A604F
:1057440070BDC04600100240FFFF7FFFFFFF3FFC1B
:10575400005C0040205C0040445C0040605C004011
:0C576400585C0040405C004000E100E0A8
:1057700070B582B0284B1B68402B45D9274B1B685E
:1057800040221A80244A1368403B1360234B1B6855
:105790001B88002B16D0224C002122481F4D036885
:1057A0001E785A1C02605A78023303601302334396
:1057B00023800234013189B22B681B8801335B10CE
:1057C0009942ECDB184B1B881B0604D5164A13883C
:1057D00016490B401380164B1B68164A1A80124B51
:1057E0001B889BB26A46D380D3889B0602D40E4B9B
:1057F000114A1A806B4606331B88DB0602D40A4B1B
:105800000E4A1A8002B070BD034B1968034A126831
:10581000118000221A60B9E714140020E814002057
:105820004060004020140020005C00400F8FFFFF0C
:10583000EC1400200084FFFFA082FFFF9082FFFF96
:1058400082B0174B1B6800221A80164B1B881B0660
:1058500004D5144A138814490B401380104B1B685D
:1058600000221A800F4B1B889BB26A46D380D388D4
:105870009B0602D40B4B0D4A1A806B4606331B88DD
:10588000DB0602D4074B0A4A1A806B4606331B8894
:105890005B0402D5034B074A1A8002B07047C0462A
:1058A000E8140020005C00400F8FFFFFA082FFFF84
:0858B0009082FFFF80C2FFFFA0
:1058B80000B583B01C4A13881C490B4013801C4B4D
:1058C8001B68052B1DD01B4B1B68002B29D1164BC1
:1058D8001B881BB2002B1EDB134B1B889BB26A462E
:1058E800D380D3889B0402D40F4B134A1A806B468B
:1058F80006331B88DB0402D40B4B104A1A8003B012
:1059080000BD0F4B1B68802213430E4A1360084BDF
:1059180000221A60D7E7044A13880B490B4013800A
:10592800DAE7FFF721FFEAE7005C00400F8FFFFF8F
:10593800181400201414002080A2FFFF8092FFFF9B
:0C594800341400204C5C00408F0F000065
:1059540082B0134B1A8813490A401A801B881B060D
:1059640004D50F4A138810490B4013800C4B1B8835
:105974009BB26A46D380D388DB0602D4084B0B4A19
:105984001A806B46DA8806331B889B0402D4044BC6
:10599400074A1A806B4606331B8802B07047C0461C
:1059A400005C00408F0F00000F8FFFFF9082FFFF0D
:0459B40080A2FFFFCF
:1059B80030B587B0B74B1B881B0500D456E1B54AF4
:1059C8001388B5490B401380B44B1B78B4490B704E
:1059D800B44B1A78B44B1A70B44B1A88B44B1A806B
:1059E8001A88120AB34802701B88DBB2B24A1370D5
:1059F800B24B1A88B24B1A80B24B1A88B24B1A8033
:105A0800B24B00221A60B24B1B68B24A1A800B785C
:105A1800212B31D0A24B1B78DBB2A12B62D0A04B3B
:105A28001A7861231A4206D09D4B1B7861221340D5
:105A3800012B00D017E1974A138897490B40138030
:105A4800994B1A78D3B2062A00D17DE0062B66D886
:105A5800002B70D0052B00D0F6E09F4B00221A6077
:105A6800FFF7EAFE924B1B887F2213409B4A136084
:105A7800964B05221A6005E18B4B1B78202B0BD027
:105A8800894B1B78222B2AD1824A138882490B40E2
:105A98001380FFF7D1FEF5E07E4B1B889BB21622E0
:105AA8006A44138013889B0402D47A4B8C4A1A8068
:105AB80016236B441B88DB0402D4764B894A1A8070
:105AC80016236B441B885B0403D5724BA0229200FB
:105AD8001A80704A13881BB2002BFBDBD2E0FFF759
:105AE80035FFCFE0704B1B78212B98D1694A13887A
:105AF80069490B401380784A07231360724B1B884F
:105B08009BB21268934204D26F4B1B889BB2724AB5
:105B18001360754B754A1A60FFF726FEB2E0092B31
:105B280000D091E06C4B00221A60FFF785FE704BA5
:105B3800FF221A60A6E0684B02221A606A4B6D4A7F
:105B48001A60FFF711FE9DE05A4B1B78012B1DD000
:105B5800584B1B78022B53D0564B1B78032B70D114
:105B6800554B1B78012B69D15B4A17331360564B91
:105B78001B889BB21268934204D2534B1B889BB27A
:105B8800554A1360584B5C4A1A6028E0524B12225F
:105B98001A605A4B1B68012B24D0594D524B1D607B
:105BA800584B1C68584A012394421DD0681E6A4607
:105BB800D11CC25CCA540133132BFAD101AB1C723D
:105BC800240A5C72514B9D4215D0514B1A7801AB97
:105BD8009A724F4A1268120ADA72434A1360FFF740
:105BE800C3FD4FE0494DD9E74A4B494A12689A42EA
:105BF800F5D00123DAE7464B1A680332D2B2E6E75A
:105C08003E4B1B68012B12D0334B43221A60364B94
:105C1800414A1A602C4B1B889BB22F4A1268934248
:105C2800DDD2294B1B889BB22B4A1360D7E72A4B3E
:105C380065221A602C4B394A1A60EBE7FFF786FE9B
:105C480020E0FFF783FE1DE0154B1B78002B02D0E8
:105C5800FFF77CFE16E00F4A13880F490B401380AC
:105C6800FFF7EAFD0EE0FFF771FE0BE0094B1B881A
:105C78009BB216226A44138013881BB2002B03DBE5
:105C8800FFF7DAFD07B030BD1388034A1340014A15
:105C98001380F5E7005C00408F0F00008060004033
:105CA8002E150020816000402F15002082600040E2
:105CB80002110020301500203115002084600040BA
:105CC8002C15002086600040921200201814002035
:105CD800EC1400200084FFFF14140020341400206A
:105CE80080A2FFFF8092FFFF201400203C70000874
:105CF8002C140020486E0008186B00082814002097
:105D0800286E0008C414002083040000586E0008A0
:105D18001C15002040570000F86F0008706F00083D
:105D2800F0B5DE4657464E464546E0B583B03C4B97
:105D38001B881B0604D53A4A13883A490B4013803E
:105D4800394C0022394FB846394B9C46BA46B946B9
:105D580033E05346374E1E6044E001AB1B882B806E
:105D68005A46354B1B681A802D4B1B889BB26A46D6
:105D7800D380D3889B0602D4294B304A1A806B46BD
:105D880006331B88DB0602D4254B2D4A1A8003B044
:105D9800F0BCBB46B246A946A046F0BD254B2349F8
:105DA8000B600232D2B26B46598801AB1B880902DC
:105DB8000B432B80402AD4D00234A51E3B682149CE
:105DC80008688342CDD0694600264E8019788B46F4
:105DD80001A95E460E80013341460B6061460968A1
:105DE8008B42B6D0531CDBB29B46402BB5D04B46FA
:105DF8001B6883420AD01878834668465E46468008
:105E080001339942CAD009490B60CAE76B465A88E0
:105E180001AB1B88120213432B805A46CCE7C046BD
:105E2800045C00400F8FFFFF02610040CC1400208B
:105E380000020020000E0020E4140020A180FFFFD3
:085E48009180FFFFD01400203F
:105E500082B0114B1B881B0604D50F4A13880F49CB
:105E60000B4013800E4B1B6800221A800A4B1B88C4
:105E70009BB26A46D380D3889B0602D4064B094A5C
:105E80001A806B4606331B88DB0602D4024B064A97
:105E90001A8002B07047C0460C5C00400F8FFFFFB5
:0C5EA000DC140020A386FFFF9386FFFFA8
:105EAC0010B5204B1B68002B34D01F4B18680028F2
:105EBC002FD01E4B1A681E4B1B689A4230D0511CB7
:105ECC001A48016014781B4A1268914225D0174A6F
:105EDC001268991A934201D2C433991A164B1B6853
:105EEC00002B11D07D290FD8134B00221A60134BB5
:105EFC001B889AB29B0402D4104B11491980D3040D
:105F0C0002D40E4B0F4A1A80FAF7D4F88020000204
:105F1C00204310BDFAF7B4FAC7E70B490160D6E786
:105F2C000020F6E7141500202C140020D4140020B7
:105F3C00D8140020040200201C140020085C00402F
:0C5F4C0082A0FFFF8290FFFFCC1100201C
:105F580070B5634B19684A1C1A60012800D1B9E072
:105F68000A788B1C5E4C2360022800D1B4E04D787F
:105F7800CB1C2360032800D1B0E08E780B1D236072
:105F88000438C0B2931E0D2B00D9A4E0052A32D0E4
:105F98000F2A30D013000C3B012B3DD904231400E9
:105FA8009C43022C5AD0C978072A7AD84D4B002234
:105FB8001A704D4B1A68541C1C6015701A684B4BAC
:105FC8001B689A4269D0484B1A68541C1C601670AA
:105FD8001A68464B1B689A4278D0434B1A68541C7F
:105FE8001C6011701A68414B1B689A4273D13E4B72
:105FF8003F4A1A606FE03B4B00221A703A4B1A680E
:10600800511C196015701A68384B1B689A4262D186
:10601800354B374A1A605EE0324B1B78AB420BD0E7
:10602800314B1A68511C196015701A682F4B1B6880
:106038009A420FD02B4B1D702B4B1A68511C1960BC
:1060480016701A68294B1B689A4244D1264B284A75
:106058001A6040E0244B264A1A60EBE7214B0022E5
:106068001A70214B1A68511C196015701A681F4B59
:106078001B689A420DD01C4B1A68511C1960167087
:106088001A681A4B1B689A4225D1174B184A1A608E
:1060980021E0154B164A1A60EDE7134B144A1A60B3
:1060A80091E7104B1B78AB428DD00F4B1A68541CEC
:1060B8001C6015701A680D4B1B689A4202D0094B78
:1060C8001D7080E7084B0A4A1A60F8E7064B084A31
:1060D8001A6082E7002070BD0020FCE70020FAE784
:1060E8002414002091120020D8140020040200205B
:0460F800CC110020A7
:1060FC0070B582B0404B1B881BB2002B11DB3F4BA1
:10610C003F4A1A603F4B1B6818783F4B1B685A007C
:10611C00D21890423FD940283DD83C4D374C2600F0
:10612C0025E0354A13883A490B401380E7E7FFF71F
:10613C000DFF14E0374B02221A600BE0364B1A6845
:10614C00511C19603168097811701A68334B1B683F
:10615C009A421CD02368013323600138C0B22A4B09
:10616C001B685A00D218904215D9402813D8012B1D
:10617C00DDD02B68022BE1D0204B1B681B78022B47
:10618C00D8D0042BDAD1234B04221A60E2E7224B3D
:10619C00234A1A60DEE7234B1A681F4B1B689A428E
:1061AC0020D99B1AC4339BB201AA13801E4B002228
:1061BC001A6001AB1B889BB27E2B18D80E4B1B8828
:1061CC009BB26A46D380D3889B0402D40A4B174AED
:1061DC001A806B4606331B88DB040BD4064B144A1F
:1061EC001A8007E09B1A9BB201AA1380DEE70E4BC4
:1061FC00FF321A6002B070BD085C0040241400200D
:10620C0000620040E014002028140020101500202B
:10621C008F0F000048140020D81400200402002026
:10622C00CC110020D41400201C14002082A0FFFFED
:04623C008290FFFF4E
:1062400000B585B0234B1A6801921B681B0429D541
:10625000019A0F2313400393019A102313400293D2
:10626000039B012B0BD0039B022B0BD0039B002B1A
:106270000ED1029B002B08D1FFF71EFB1DE0FFF79C
:1062800053FD1AE0FFF73AFF17E0FFF795FB14E024
:10629000039B032B11D1104B1B68002B0DD1FFF773
:1062A000D7FD0AE00B4B1B685B0508D4094B1B6844
:1062B0001B050AD5074B094A1A6005B000BDFFF758
:1062C0000FF9044B064A1A60F7E7024B054A1A60B9
:1062D000F3E7C046445C004028140020FFF7FFFFAE
:0862E000FFFBFFFF7F800000BF
:1062E80070B5134B1B68002B21D0124B1A68511C38
:1062F800196010701A68104B1B689A4204D00F4E30
:106308000C4DAC24A4000AE00A4B0D4A1A60F6E7CB
:10631800C02189008C466344991AA14207D9FAF72B
:10632800B1F832682B68991A9A42F6D9F0E770BD2D
:106338002C140020D014002000020020CC140020CF
:04634800000E002023
:10634C00074B1B68002B00DBFEE7054A1168802316
:10635C001B060B4313608369023383617047C0468D
:04636C002CED00E034
:10637000555342206173207669727475616C2043B5
:046380004F4D3D0040
:1063840043466F72746820666F722053544D3332E3
:106394004630343220762E002028632932303230C1
:1063A4002D323420572E536368656D6D6572740009
:0863B400202D3E444247200069
:0863BC004B65726E656C3A003E
:1063C400B0300008063100087A3100087A3100083C
:1063D400183100082A3100083C31000868310008EF
:1063E400537461636B3D00002052657475726E00D6
:1063F40020557365723D000020436F6465546872D4
:106404006561643D00000000456D70747900000012
:10641400466C6173680000005F50726F6A65637454
:10642400206C6F61646564002020204155544F4501
:1064340058453D002852533233323D5465726D69DC
:106444006E616C29000000005350493D00000000BB
:10645400202054696D65723A467265713D000000F2
:10646400487A2050574D313D000000002020204D37
:106474004F543A00537465703D0000006D73204E14
:106484005354503D0000000044432F50574D3100F9
:1064940020636F6E6669726D20772E7570706572F9
:1064A4002063617365202759270000002063616E13
:0864B40063656C6C6564200057
:1064BC00205761726E3A2077696C6C206F7665722A
:1064CC0072696465204B65726E656C204F50207745
:0C64DC002E73616D65206E616D652000FF
:1064E800536176652061637475616C20776F726B98
:0C64F80020696E20466C617368203F0034
:10650400313238205352414D2062797465732073BF
:1065140074617274696E672066726F6D20307800E2
:106524000000000000000000000000000000000067
:106534000000000000000000000000000000000057
:106544000000000000000000000000000000000047
:106554000000000000000000000000000000000037
:106564000000000000000000000000000000000027
:106574000000000000000000000000000000000017
:106584000000000000000000000000000000000007
:1065940000000000000000000000000000000000F7
:1065A40000000000000000000000000000000100E6
:1065B40000000500000000000000000000000000D2
:1065C40000000000000000000000000000000100C6
:1065D40000000400000004000000000000000000AF
:1065E40000000000000000000000010000000000A6
:1065F4000000000000000000000000000000000097
:10660400000004000000040000000400000000007A
:106614000000000000000000000000000000000076
:106624000000000000000000000000000000000066
:106634000000040000000000000005000000050048
:106644000000050000000400000004000000040035
:106654000000040000000000000001000000010030
:10666400000001000000010000000300000003001E
:10667400000003000000030000000300000003000A
:1066840000000300000003000000030000000300FA
:1066940000000300000003000000020000000200EC
:1066A40000000200000002000000020000000100DF
:1066B40000000100000008000000080000000800BD
:1066C40000000800000008000000080000000800A6
:1066D4000000080000000800000008000000080096
:1066E4000000080000000800000008000000080086
:1066F4000000080000000800000002000000020082
:106704000000010000000100000001000000010081
:0C67140000000500000001000000010072
:106720004552524F5200000044524F5000000000AA
:106730004455500000000000535741500000000035
:106740004F56455200000000524F54000000000018
:106750002D524F54000000005049434B00000000F0
:10676000524F4C4C00000000494E4A454354000033
:106770002B00000000000000312B00000000000092
:106780002D00000000000000312D0000000000007E
:1067900041425300000000005348494654000000A5
:1067A000414E4400000000004F5200000000000075
:1067B000584F5200000000004E4F540000000000EF
:1067C0002B2F2D00000000002A0000000000000018
:1067D0002F000000000000002A2F00000000000031
:1067E0004D4F4400000000002F4D4F4400000000BA
:1067F00052414E444F4D00003D3D0000000000005E
:10680000213D0000000000003E00000000000000EC
:106810003E3D0000000000003C00000000000000C1
:10682000553C0000000000003E3D0000000000005C
:10683000303D000000000000564152434F4E000022
:1068400052455600000000004B45593F0000000033
:106850004B45590000000000454D49540000000020
:106860002E000000000000002E4800000000000084
:106870002E440000000000002E2200000000000056
:10688000445A0000000000004858000000000000CA
:1068900052583F0000000000525800000000000065
:1068A00054580000000000004E5458000000000042
:1068B0005458220000000000584E4F5000000000C5
:1068C0004D53000000000000445300000000000091
:1068D000544958000000000054494D450000000094
:1068E000465245510000000050574D310000000055
:1068F0004D4F5400000000004F4800000000000011
:106900004F4C0000000000004950550000000000FE
:106910004950440000000000495A000000000000F7
:106920005244494E00000000524144430000000020
:10693000494E492D53504900535049000000000072
:106940002E5300000000000046530000000000002D
:106950004F50530000000000555345520000000006
:1069600053454500000000004D454D00000000006B
:10697000535400000000000052554E00000000007B
:106980004E4F2D4442470000444542554700000009
:10699000464F52474554000041424F5254000000B8
:1069A0005245504C41434500524553544F524500C7
:1069B000494600000000000043415345000000002C
:1069C0003C434153450000003E4341534500000015
:1069D000454C5345000000005448454E000000005F
:1069E000444F000000000000554E54494C00000088
:1069F0005748494C45000000414741494E000000BE
:106A0000464F5200000000004C4F4F500000000065
:106A10004900000000000000434F4E5449000000B0
:106A2000425245414B0000005A425245414B000042
:106A300052455455524E00003A000000000000003C
:106A40003B00000000000000646F5354520000003F
:106A5000646F494F53545200646F4C495400000016
:106A6000646F4C4954384200646F56414C554500A0
:106A7000646F524556000000646F494600000000F4
:106A8000646F434153450000646F3C4341534500EC
:106A9000646F3E4341534500646F454C53450000CD
:106AA000646F444F00000000646F554E54494C0021
:106AB000646F5748494C4500646F414741494E0057
:106AC000646F464F520000004C4F4F5000000000D2
:106AD00052502D310000000052502D3400000000B3
:106AE0004155544F4558450042415544000000006F
:106AF00053504C495400000056494450494400004A
:106B00003F00000000000000534156450000000017
:086B10004C4F4144000000005D
:106B18001803430046006F007200740068002D00DF
:086B28004D0049004400490042
:106B3000FEE7FEE7FEE7FEE7FEE7FEE7FEE7FEE72D
:106B4000FEE7FEE7FEE7FEE7FEE7FEE7FEE7FEE71D
:106B5000FEE7FEE7FEE7FEE7FEE7FEE7FEE7FEE70D
:106B6000FEE7FEE7FEE7FEE7FEE7FEE7FEE7FEE7FD
:106B7000FEE7FEE7FEE7FEE7FEE7FEE7FEE7FEE7ED
:106B8000FEE703488546FEF725FC03E0704700005A
:046B900000180020C9
:106B940011488546114C20680434004201D08047D6
:106BA400F9E70F480F49091A082903DB002202609C
:106BB400043001600C480D49884205D00268043055
:106BC40003B4904703BCF7E700208646EC46002058
:106BD4000021074A9047FEE700180020987100083A
:106BE4003815002080160020816E0008816E000890
:046BF400810B000809
:106BF80004207146084202D1EFF3088001E0EFF368
:0C6C080009800149084700004D630008A6
:106C1400756E646572666C6F77212000202D2D2DB2
:026C240020004E
:106C260010B502003030C0B2392801D93732D0B29F
:066C3600F9F7E9FA10BDB8
:066C3C002849502D3E0026
:106C420010B5441C0078002806D0F9F7DEFA0134AA
:0A6C5200631E18780028F8D110BD69
:106C5C0063616E277420534545204B65726E656CDD
:106C6C004F707300557365724865616465725F534C
:106C7C0074727563743D0000566172436F6E3A56C0
:066C8C00616C75653D001E
:106C920010B5040003061B0F18003030392801D943
:106CA20037331800F9F7B1FA0F20044020003030D2
:106CB200392800D90730F9F7A8FA2020F9F7A5FA00
:026CC20010BD03
:106CC4004572726F722300002028636F6C200000ED
:106CD400206E6F7420666F756E6400005F53796E6A
:106CE40074617820457272005F537461636B204550
:106CF400727200005F436F6D70696C65206F6E6C1B
:106D0400790000005F4E6F20492F4F20436F6D6D57
:106D140020416363657373005F496E76616C6964D7
:106D240020436F6465206163636573730000000032
:106D34005F6F7574206F6620436F6E74657874009E
:106D44005F52756E74696D65206F6E6C790000001A
:106D54005F5468726561642063616E63656C6C6521
:106D6400640000005F4E756D626572206F7574205B
:106D74006F662052616E6765000000005F446976AB
:106D84002E6279205A65726F000000002020636F24
:0A6D94006D70696C696E672E2E00A9
:0E6D9E0010B5F9F7F4FD2020F9F731FA10BD19
:0A6DAC0042617564526174653D0098
:106DB6002F280FD90300303BDBB2092B08D90A294B
:106DC6000BD00300413B052B0AD83738C0B27047B9
:106DD6001800FCE701204042F9E701204042F6E7AF
:066DE60001204042F3E72A
:0E6DEC0042617564206368616E676521200056
:0A6DFA0010B50120FBF7F7FC10BDF7
:106E04005553415254205465726D696E616C20670C
:0A6E1400657473206C6F7374210025
:0A6E1E0010B50020FBF7E5FC10BDE5
:106E280012010002000000408304405724050000BE
:026E3800000157
:0E6E3A0010B56B20FBF72BFAFCF7D9FB10BD4F
:026E4800000048
:0E6E4A0010B56C20FBF723FAFCF7D1FB10BD4E
:106E5800120100020000004083044357240500018A
:026E6800000127
:0E6E6A0010B56D20FBF713FAFCF7C1FB10BD4D
:096E780028566172436F6E3D0063
:0E6E820010B56E20FBF707FAFCF7B5FB10BD4C
:106E9000203C2D6E6F742061204B65726E656C20F6
:106EA0004F50206E6F722061206E756D62657200AA
:106EB000203C2D696E76616C696420666F72204299
:106EC00061636B2D4374726C00000000203C2D52F6
:0D6ED000756E74696D65204572726F7200F9
:0E6EDE0010B57120FBF7D9F9FCF79BFB10BD36
:106EEC0020202841444320696E6974292000000049
:0D6EFC00202028414443206F6666292000B5
:0E6F0A0010B57220FBF7C3F9FCF785FB10BD34
:106F18002064656275672066696E697368656420B8
:016F28000068
:0E6F2A0010B57320FBF7B3F9FCF775FB10BD33
:106F38004C6F616420466C6173682050726F6A659B
:106F48006374203F000000004C6F616420456D7041
:0D6F580074792050726F6A656374203F00E9
:0A6F660010B50120FDF7E5FB10BD9A
:106F700009026500020100803109040000000101DE
:106F800000000924010001090001010904010002B7
:106F90000103000007240100014100062402010151
:106FA0000006240202020009240301030102010079
:106FB00009240302040101010009058102400000C7
:106FC0000000052501010309050202400000000040
:056FD00005250101018F
:0A6FD60010B50020FDF7ADFB10BD63
:076FE0006E6F2055534200C3
:0F6FE800564944203D200000504944203D2000E0
:106FF8000902430002010080310904000001020275
:1070080000000524001001052401030004240207E0
:107018000524060001070583031000400904010048
:10702800020A00000007058102400000070502026D
:0370380040000015
:07703C0000C2010000000882
:107044000A0010D00300400800E052008242FCD93C
:10705400002000E05208934200D39B1A40418A4228
:0A706400F8D11900704700207047B2
:10706E0010B50400000F16D12001000F17D1200219
:10707E00000F18D12003000F19D12004000F1AD1D0
:10708E002005000F1BD12006000F1CD10F20204021
:10709E00FFF7C2FD10BDFFF7BFFD2001000FFFF788
:1070AE00BBFD2002000FFFF7B7FD2003000FFFF717
:1070BE00B3FD2004000FFFF7AFFD2005000FFFF713
:0C70CE00ABFD2006000FFFF7A7FDDFE779
:1070DA0010B504003020F9F794F87820F9F791F800
:0870EA002000FFF7BFFF10BDFD
:1070F200CA1751408B1A17D0C1174A4004B44840EE
:10710200411A48081A0000E052008242FCD90020CD
:1071120000E05208914200D3891A40419A42F8D1C4
:0C71220004BC5040801A704700207047E9
:10712E000A000FD00300400800E052008242FCD952
:10713E00002000E05208934200D39B1A40418A423D
:08714E00F8D1704700207047E2
:10715600CA1751408B1A19D0C11706B44840411AB4
:1071660048081A0000E052008242FCD9002000E0E4
:107176005208914200D3891A40419A42F8D10CBC78
:1071860053405840C01A5140891A70470020704732
:10719800C97300081002002024130000DF730008E0
:1071A80000000020B8710008100200000000000074
:1071B800E50E0008F50E00081D0F00084D0F000829
:1071C800650F0008790F00089D0F0008C10F00081F
:1071D8000110000861100008C1100008DD10000847
:1071E800ED100008091100081911000831110008F4
:1071F8007911000895110008B1110008CD11000897
:10720800DD110008ED1100080912000841120008FC
:1072180079120008B1120008F112000809130008D9
:10722800291300085D13000881130008A51300083E
:10723800C9130008E913000849130008D94D0008CC
:10724800F5500008092700088919000839190008AD
:10725800E51900082D1A0008151C0008FB6D000828
:107268000D1400082D1400084D140008352C0008D2
:107278002D1C0008551C00081F6E0008A1140008EA
:10728800792C0008A92C0008C9140008E514000886
:107298009D510008D15100081D520008912D000889
:1072A800012E0008712E0008D52E0008392F00087D
:1072B800112D00082D3000083932000875320008F9
:1072C8004D1A000801160008A91C0008111B000827
:1072D800613D000809530008211600082D16000812
:1072E8003916000851190008F140000869410008E2
:1072F8005D460008E94600083B6E00084B6E000832
:107308006B6E0008836E00087D24000805150008D0
:10731800C5240008DF6E00080B6F00082B6F0008FB
:10732800F12400081D2500083915000881170008F8
:10733800551500086915000891150008214E000828
:1073480075250008676F0008D76F00084516000804
:1073580085160008A5160008D11600089D470008E4
:10736800C9470008F947000829480008FD16000821
:1073780021170008B1170008E9170008511700087D
:10738800211800087118000819190008291900089F
:1073980041220008654E0008F94E0008814F000898
:1073A800ED480008F94F00083550000801000000BA
:1073B8000011002090120020C8110020006CDC028F
:1073C800206861680834094204D000220270013044
:0673D8000139FBD17047F2
:1073DE0020686168A2680C34124205D00B780370E5
:0A73EE0001300131013AF9D1704776
:0400000508006B8301
:00000001FF
